:100000000C9458000C9477000C9477000C947700B3
:100010000C9477000C9477000C9477000C94770084
:100020000C9477000C9477000C9477000C94770074
:100030000C9425310C9477000C9477000C94CB3100
:100040000C9427010C9477000C9477000C947700A3
:100050000C948F010C9477000C9483010C9477001E
:100060000C9477000C9477000C9477000C94770034
:100070000C94CD010C9477000C94C1010C94770082
:100080000C9477000C9477000C9477004F6E6C6999
:100090006E650A000A2A2A2A2A2A2A2A426F6F74BF
:1000A000696E672025732A2A2A2A2A2A2A0A00002A
:1000B00011241FBECFEFD0E4DEBFCDBF13E0A0E020
:1000C000B1E0E8EDF1EA00E00BBF02C007900D924D
:1000D000A230B107D9F718E2A2E0B3E001C01D9247
:1000E000AF30B107E1F70E94B8000C94EA500C94CD
:1000F0000000FC011182108283E0089580E06CE032
:1001000046E00E94FF0180E060E579E20E947B0208
:1001100081E068E046E00E94FF0181E00E94B102B8
:100120000E94BD0000D000D084E990E0EDB7FEB79A
:100130009283818387E291E0948383830E943F4D81
:100140000F900F900F900F900E94C0060E94EF0733
:100150008DE191E00E940C0800D08CE890E0EDB7B2
:10016000FEB7928381830E943F4D0F900F900895B8
:100170000E947E000E94D006FDCFF8941092B60037
:1001800016BC8EE387BD92E094BD85E085BD85B346
:1001900085BB90936E00109203031092020380912E
:1001A00002039091030390930503809304037894D2
:1001B00008952091020330910303809102039091EE
:1001C000030328173907A9F7C901089507C022E3D7
:1001D00030E0000021503040E1F701970097B9F777
:1001E0000895BC01409102035091030380910203E2
:1001F0009091030348175907A9F720910203309102
:100200000303809102039091030328173907A9F78C
:10021000241B350B2617370780F308950895209186
:100220000603309107034091080350910903809120
:10023000060390910703A0910803B09109032817C2
:1002400039074A075B0759F7B901CA0108951F9298
:100250000F920FB60F920BB60F9211242F933F936C
:100260004F935F936F937F938F939F93AF93BF93BE
:10027000EF93FF9380910203909103030196909373
:100280000303809302038091040390910503019678
:1002900090930503809304038091040390910503D8
:1002A0008D379105B9F410920503109204038091E3
:1002B000060390910703A0910803B09109030196EA
:1002C000A11DB11D8093060390930703A09308031B
:1002D000B09309030E943308892B11F00E94B208E1
:1002E000FF91EF91BF91AF919F918F917F916F910E
:1002F0005F914F913F912F910F900BBE0F900FBECA
:100300000F901F9018951F920F920FB60F92112405
:10031000109255010F900FBE0F901F9018951F92CD
:100320000F920FB60F920BB60F9211242F933F939B
:100330004F935F936F937F938F939F93AF93BF93ED
:10034000EF93FF93E0914B01F0914C018081E0919C
:100350005601F0915701309709F00995FF91EF91FF
:10036000BF91AF919F918F917F916F915F914F91CD
:100370003F912F910F900BBE0F900FBE0F901F90CB
:1003800018951F920F920FB60F92112410926201CE
:100390000F900FBE0F901F9018951F920F920FB6DF
:1003A0000F920BB60F9211242F933F934F935F93AD
:1003B0006F937F938F939F93AF93BF93EF93FF932D
:1003C000E0915801F09159018081E0916301F09131
:1003D0006401309709F00995FF91EF91BF91AF91BA
:1003E0009F918F917F916F915F914F913F912F914D
:1003F0000F900BBE0F900FBE0F901F90189590E0BE
:100400002DE030E0829FF001839FF00D929FF00D70
:100410001124E55BFE4FA281B3811C92A481B581BA
:100420006C93A681B78188ED8C93A085B1854C93A0
:100430001286148613860895CF93DF93AB0190E064
:100440002DE030E0829FD001839FB00D929FB00DD0
:100450001124A55BBE4FED012A9691E00AC0988356
:10046000ED91FC911197808388818823E9F74F5F94
:100470005F4FFA018491882391F7DF91CF9108951E
:10048000CF93DF93EB0190E02DE030E0829FD0012D
:10049000839FB00D929FB00D1124A55BBE4F9D01AF
:1004A000265F3F4F91E00BC0F9019083ED91FC91E5
:1004B00011978083F90180818823E1F72196888153
:1004C000882391F7DF91CF91089590E02DE030E0FF
:1004D000829FF001839FF00D929FF00D1124E55B48
:1004E000FE4F81E08287A081B1816C933A96808132
:1004F0008823E9F7089590E02DE030E0829FF00135
:10050000839FF00D929FF00D1124E55BFE4F7487E1
:100510006387089591E090935501E0914B01F0912C
:100520004C018083809155018823E1F70895209143
:100530000A0330E04DE050E0249FF001259FF00DCC
:10054000349FF00D1124E55BFE4F91E09287A0816E
:10055000B1818C933A9680818823E9F780E090E01E
:10056000089580930A038DE391E090930C28809383
:100570000B280895DF93CF93CDB7DEB7FE013896F1
:100580008BE093E060E470E04E815F819F010E9408
:10059000894D4BE053E08D8190E02DE030E0829F6B
:1005A000D001839FB00D929FB00D1124A55BBE4F6B
:1005B0009D01265F3F4F91E00CC0F9019083ED91C2
:1005C000FC9111978083F90180818823E1F74F5FC7
:1005D0005F4FFA018081882381F7CF91DF910895E1
:1005E0009C01F999FECF32BD21BDF89A80B50895DE
:1005F00020E090915D0380915E03981321E0822FAB
:100600000895CF93DF93EC0140915D03E42FF0E078
:10061000CF0101966AE070E00E94635020915E0372
:1006200030E082179307A9F088819981AA81BB8164
:10063000EE0FFF1FEE0FFF1FE35AFC4F82839383E1
:10064000A483B583842F8F5F8A3008F080E0809385
:100650005D03DF91CF910895DF93CF930F92CDB7D4
:10066000DEB780915E038983298189818F5F8983C9
:1006700089818A3008F01982898180935E0330E095
:10068000220F331F220F331F215A3C4FC9010F90F5
:10069000CF91DF9108959093E2208093E120089517
:1006A00081E090E0089581E090E0089585E691E092
:1006B000089580915B0390915C0308958DE493E02D
:1006C0000895AC01615020E00CC0DA01A20FB11D09
:1006D0009C91FA01E60FF11D80818C93908361500B
:1006E0002F5F261790F308950F931F93DF93CF93F7
:1006F0000F92CDB7DEB78823E9F10FEF1FEF10930C
:10070000C7210093C6210E94EB4C60E071E00E947B
:100710006350809309228DEC9BEA9093F52180939E
:10072000F4219093BB218093BA211093C5210093AB
:10073000C4218FB78983F8948CEB91E260E070E07C
:1007400048E050E020EF32E00E94234D20E037E007
:10075000A22FB0E0A454BE4D9C91E32FE21BF0E029
:10076000E454FE4D80818C9390832F5F243081F779
:1007700089818FBF0F90CF91DF911F910F910895C5
:10078000CF92DF92EF92FF921F93DF93CF93CDB77B
:10079000DEB7AB970FB6F894DEBF0FBECDBF80EBD0
:1007A00096E30197F1F782E00E944E368093B921DB
:1007B0008C81807E81608C8382E10E944E3620E0B5
:1007C000892B09F021E02295220F207E8C818F79E0
:1007D000822B8C839D819F7C809109228E838F5FE9
:1007E00080930922906C9D83E091D221F091D321D6
:1007F000099598878F8385E10E9457366EEE71E0E8
:100800000E94AA37892B59F08D81837F88608D8360
:100810008FEF9FEF98878F839A87898722C085E122
:100820000E945736DE011996FC0188E001900D9276
:100830008150E1F7AE01475F5F4F20E037E0DA011A
:10084000A20FB11D9C91832F821BFA01E80FF11DAD
:1008500080818C9390832F5F243089F78D818C6009
:100860008D83E091D621F091D72109959A8B898BC0
:10087000E091DE21F091DF2109952B8B3C8B4D8B94
:100880005E8B6F8B788F898F9A8F0E942D368BA706
:100890000E94FF359AA789A7CE010496BE016F5F1B
:1008A0007F4F0E94B43213E068ECE62EF12C50E248
:1008B000C52E5EE4D52E69817A818B810E94982DA8
:1008C0008034910519F421E030E020C08434910592
:1008D000D9F4133021F4C6010197F1F713C0123097
:1008E00041F484EF91E0F7013197F1F70197D9F7DF
:1008F00009C0113039F480ED97E0F7013197F1F735
:100900000197D9F71150B9F620E030E0C901AB9654
:100910000FB6F894DEBF0FBECDBFCF91DF911F9110
:10092000FF90EF90DF90CF90089580914B039091CE
:100930004C03892B09F467C00E949036E0915B0359
:10094000F0915C0360898685978570E00E9473371B
:10095000E0915B03F0915C03808990E00E94FA359E
:10096000E0915B03F0915C03A7E8B3E02681378157
:10097000C901FC0188E001900D928150E1F7E091FE
:100980005B03F0915C03AFE8B3E022853385C901D6
:10099000FC0188E001900D928150E1F720E037E002
:1009A000A22FB0E0A957BC4F9C91E32FE21BF0E0CF
:1009B000E957FC4F80818C9390832F5F243081F71F
:1009C00020E037E0A22FB0E0A157BC4F9C91E32F6D
:1009D000E21BF0E0E157FC4F80818C9390832F5F06
:1009E000243081F785E167E873E00E94623684E194
:1009F0006FE873E00E946236E0914B03F0914C0384
:100A00008DE493E0099508950E949036E0915B0390
:100A1000F0915C0360898685978570E00E9473374A
:100A2000E0915B03F0915C03808990E00E94FA35CD
:100A3000E0915B03F0915C03A7E8B3E02681378186
:100A4000C901FC0188E001900D928150E1F7E0912D
:100A50005B03F0915C03AFE8B3E022853385C90105
:100A6000FC0188E001900D928150E1F720E037E031
:100A7000A22FB0E0A957BC4F9C91E32FE21BF0E0FE
:100A8000E957FC4F80818C9390832F5F243081F74E
:100A900020E037E0A22FB0E0A157BC4F9C91E32F9C
:100AA000E21BF0E0E157FC4F80818C9390832F5F35
:100AB000243081F785E167E873E00E94623684E1C3
:100AC0006FE873E00E946236E091E120F091E2204D
:100AD0008DE493E009950895DF93CF930F92CDB7FE
:100AE000DEB790915E0380915D038917A1F1998330
:100AF0008981E82FF0E0EE0FFF1FEE0FFF1FE15A94
:100B0000FC4F89818F5F898389818A3008F019823F
:100B1000898180935E033097F1F0808191814097C5
:100B2000D1F40280F381E02DF0935C03E0935B034A
:100B30000190F081E02D80818770813019F40E944E
:100B4000040502C00E949504E0915B03F0915C03F0
:100B500087898D7F878B0F90CF91DF91089580E0FB
:100B600060E070E00E946C050895FF920F931F9360
:100B7000CF93DF938C01F62EEA0122E8621711F47D
:100B80000E94AF05F80180819181009729F0855876
:100B9000924009F04FC049C080E060E070E040E062
:100BA00050E020E030E00E94FB2DF999FECF89E073
:100BB00090E092BD81BDF89A20B5F999FECF8AE008
:100BC00090E092BD81BDF89A90B5822F8B50803114
:100BD00010F49095291328E1822F0E94432D81E083
:100BE0000E942C2A88E00E94D92B0E94FB338BE4C0
:100BF00093E0909356038093550380EC93E0909399
:100C00005203809351038DE493E00E94691E88ECA7
:100C100091E20E940A3586E10E94D92B85E892E094
:100C2000F8019183808381E009C08F2DBE010E946D
:100C30006C05F4CFF8011182108283E0DF91CF912F
:100C40001F910F91FF9008958091A3038F5F809370
:100C5000A303815008951F93CF93DF93EC01162FC8
:100C6000888580FF1CC0EC81FD813097C1F0D09356
:100C70009A03C093990382E08887CE01069609956E
:100C8000992787FD90950297029710F0133829F461
:100C9000CE01BE010E94530602C081E08887DF9129
:100CA000CF911F910895CF92DF92EF92FF920F9311
:100CB0001F93CF93DF938C017B01C0909903D09059
:100CC0009A03DC0118968C911897882341F11896A5
:100CD0001C92C0919703D09198030BC00C171D076D
:100CE00029F0CE0167E8A8010E942B060990D8815F
:100CF000C02D209799F7D8011496ED91FC91159786
:100D0000309769F00E151F0551F010939A03009368
:100D10009903C801069663E840E050E00995E09128
:100D20009703F09198030E171F07A1F4F801808133
:100D3000918190939803809397030EC08081918155
:100D40008017910731F4D8018D919C919183808314
:100D500003C0FC01309791F7D0929A03C092990397
:100D6000DF91CF911F910F91FF90EF90DF90CF9087
:100D700008956091990370919A030E945306089513
:100D80008AE88093A3031092A5031092A403109203
:100D900098031092970310929A0310929903089562
:100DA0001F93CF93DF93809146048823C1F0109264
:100DB0004604C0919703D091980311E00EC0898535
:100DC000882341F018871986CE0162E840E050E0A0
:100DD0000E942B060990D881C02D209781F7209181
:100DE000A403222309F470C08091A50390E0FC01C4
:100DF000EE0FFF1FEE0FFF1FE80FF91FEA55FC4F24
:100E000060816093A203418152815093A10340937A
:100E1000A0030380F481E02DF0939F03E0939E03F1
:100E200001968F7190708093A50321502093A403A5
:100E3000309709F042C08091970390919803909366
:100E40009D0380939C0311E031C080914604882368
:100E5000B9F010924604C0919703D09198030EC048
:100E60008985882341F018871986CE0162E840E021
:100E700050E00E942B060990D881C02D209781F761
:100E80004091A0035091A10380919C0390919D03F8
:100E90006091A2030E942B06E0919C03F0919D03B8
:100EA0008081918190939D0380939C0380919C030A
:100EB00090919D03892B49F607C0613811F481E0B8
:100EC0008087CF010E942B06809146042091A403C5
:100ED00030E0280F311DC901DF91CF911F91089596
:100EE000809146042091A40330E0280F311DC901F0
:100EF0000895DC012091A403203219F421E030E0B0
:100F00001AC08091A503820F8F7180939B0390E09C
:100F1000FC01EE0FFF1FEE0FFF1FE80FF91FEA5550
:100F2000FC4F608352834183B483A3832F5F20935C
:100F3000A40320E030E0C90108950F931F930091AE
:100F4000990310919A030E942B0610939A03009321
:100F500099031F910F910895CF93DF93DC01EB016B
:100F60006091970340919803862F942F9C01F9017B
:100F700003C00190F081E02DEA17FB07B9F030972C
:100F8000C1F76C9311964C931197B0939803A0936B
:100F9000970381E018968C93189717961C921E92CF
:100FA0001697CD0161E8AE010E949D07DF91CF91B8
:100FB0000895FC01009741F080858150823020F433
:100FC00081E0818780934604089520E030E0FC01B1
:100FD0008085882311F021E030E0C9010895CF9386
:100FE000DF93C3E3D1E004C060E070E00E94AC078F
:100FF000899199910097C1F7DF91CF910895CF938F
:10100000DF93EC0102C00E94B90689919991009783
:10101000D1F7DF91CF910895CF93DF93EC0104C016
:1010200060E070E00E94AC07899199910097C1F748
:10103000DF91CF91089520E030E0FC018681978117
:10104000892B11F421E030E0C9010895FC012281CF
:10105000338180819181280F391FC9010895FC01D6
:101060008081918108952091470430914804211591
:10107000310511F021E030E0C90108958091470465
:1010800090914804892B19F420E030E004C02091AD
:10109000490430914A04C901089580914704909110
:1010A0004804892B29F410924A04109249040895A7
:1010B0000E94D900BC01E0914704F09148044281AC
:1010C000538180819181480F591F461B570B0CC0DB
:1010D0002281338180819181280F391F261B370B94
:1010E0002417350708F4A9010480F581E02D309715
:1010F00079F7460F571F50934A04409349040895C7
:10110000CF93DF93EC01E0914704F09148048E17F0
:101110009F0741F48C819D819093480480934704FC
:1011200014C0FC01309731F0848195818C179D07A4
:10113000C1F707C01D821C821F821E82DF91CF91E2
:1011400008958C819D81958384830E944D08F2CF00
:10115000FC0180819181860F971F918380830E947B
:101160004D0808958EE991E00E94D9070895EF9205
:10117000FF920F931F93CF93DF937C01FC0180813B
:101180009181009729F08A35910509F06DC00BC057
:1011900010924804109247048AE590E0F701918389
:1011A000808381E065C0673849F59A01E091470482
:1011B000F091480403C00480F581E02D309741F39D
:1011C0008681978182179307B1F3E0934704F093E8
:1011D00048040FC016968D919C911797821793071C
:1011E00011F0FD0106C014968D919C911597958381
:1011F0008483A481B581109769F7CECF623861F6F8
:10120000C0914704D091480400E010E02AC0CE010C
:101210000E94F337892B01F18E819F8168E8AE012E
:101220000E947907892BA1F41F821E828C819D81E7
:101230000115110521F0F8019583848304C0909372
:101240004804809347041D821C820E944D08D8CF19
:101250008EE991E00E94D9078E018C819D819C01CD
:10126000E9012097A1F698CFF7011182108283E05F
:10127000DF91CF911F910F91FF90EF900895CF9341
:10128000DF93EC018EE991E00E94D9078E819F8166
:10129000892B69F0E0914704F091480406C0EC17EF
:1012A000FD07A9F00480F581E02D3097C1F780910A
:1012B000990390919A039F838E8380914704909124
:1012C00048049D838C83D0934804C09347040E94B4
:1012D0004D08DF91CF9108950F931F938C010E94C9
:1012E0000A38C8010E943F091F910F9108950F937A
:1012F0001F938C010E94D437C8010E943F091F919F
:101300000F9108950F931F938C010E941538C80107
:101310000E943F091F910F910895E0916204F0919E
:101320006304309711F480E008950995089590932F
:101330006304809362040895FC0180919903909165
:101340009A0391A780A773A762A70895FC018091D3
:10135000990390919A03968B858B708F678B089574
:101360009C018091CB229091CC22892B11F081E0BD
:1013700008958091990390919A039093CC22809341
:10138000CB223093CE222093CD2280E00895AC0171
:1013900010924F046091990370919A03E8E5F4E08C
:1013A00020E014C0808191818417950769F48281BF
:1013B00093818617970741F420934F04118210827E
:1013C000CA010E942F3A089534962F5F223050F3BD
:1013D00020934F040895CF93DF93A0917122B09191
:1013E0007222109719F0ED01A89605C0C0916D22E8
:1013F000D0916E22659680916A2286FF2AC0109253
:101400004D04E8E5F4E040E016C0208131815096BB
:101410008D919C9151972817390759F482819381B6
:10142000009739F040934D04998388831B821A8278
:1014300006C034964F5F423040F340934D0480E540
:1014400094E00E941B08892B21F080E594E00E9423
:101450006C0988819981009731F04A815B816091A4
:10146000E3200E949D07DF91CF91089585EB91E0E5
:1014700062E040E050E00E949D0710925B221092D3
:101480005A221092C5200895682F8091CB22909106
:10149000CC2240E050E00E949D070895AC0185EB0E
:1014A00091E060E00E9479070895AC0185EB91E03E
:1014B00061E00E9479070895EF92FF920F931F93C6
:1014C000CF93DF9380915A2290915B22009709F489
:1014D0000BC18150954008F0F8C08091EB229091AB
:1014E000EC22892B59F58091ED229091EE22892BE7
:1014F00029F58091EF229091F022892BF9F48091C7
:10150000F1229091F222892BC9F48091F3229091DB
:10151000F422892B99F48091F5229091F622892B5F
:1015200069F48091F7229091F822892B39F4809107
:10153000F9229091FA22892B09F4C7C08091EB22FD
:101540008F3F09F4C7C08BEE92E20E94E710882318
:1015500031F08BEE92E20E941C11EC0108C00E9457
:10156000EA0DFC01009709F4B0C0C081D181209739
:1015700039F0898D9A8D8530910509F04CC00BC0EA
:101580008BEE92E260E070E040E020E030E00E940C
:101590005D11EC0102C01A8E198E9E01235D3F4F32
:1015A00003ED12E240915A2250915B22C901B80129
:1015B0000E94084DC35DDA4F80915A228883CD5234
:1015C000D540C801089660E840E050E00E94B01B9A
:1015D000892B19F0C801089602C080E090E060E015
:1015E00070E0AE010E945B166091F9207091FA20C4
:1015F0008091FB209091FC2028EE33E040E050E009
:101600000E947650CE018396BA01A9010E949138BA
:1016100081E08BA75FC0009799F49E01235D3F4F47
:10162000E3EDF2E240915A2250915B22C901BF01E1
:101630000E94084DC35DDA4F80915A22888345C0CD
:10164000029761F483E090E09A8F898FCE014B96E8
:1016500045E050E060E070E00E9491386091F92030
:101660007091FA208091FB209091FC2028EE33E0CD
:1016700040E050E00E947650CE018396BA01A90165
:101680000E94913880E1E82EF12CEC0EFD1EC7017E
:101690000E948D098E01035D1A4FD801EC91EE2353
:1016A000A1F0E0935A2210925B2223ED32E2AE01C8
:1016B000435D5F4FC901BA014E2F50E00E94084DB3
:1016C000F8011082C7010E948D0910925B221092CE
:1016D0005A220AC080E090E00E948D0910925B229D
:1016E00010925A221092C520DF91CF911F910F9135
:1016F000FF90EF900895DF92EF92FF920F931F9368
:10170000CF93DF937C018A01FC0180819181009756
:1017100029F08C5E924009F023C12CC080E00BC000
:10172000E82FF0E0EE0FFF1FEE0FFF1FE85AFB4F10
:10173000118210828F5F823098F380934B048091E6
:10174000990390919A0390936104809360040E949E
:1017500024068093E32080E594E06EE370E00E942D
:1017600082090E9417448CEE92E0F70191838083F6
:1017700081E0FAC0623009F4DFC0633030F46623E0
:1017800009F4B3C0613079F7C9C0673819F0683817
:1017900051F73CC010924C04C8E5D4E013C08A81D4
:1017A0009B818017910741F4888199810E942F3A8B
:1017B000198218821B821A82249680914C048F5FB2
:1017C00080934C0480914C04823048F3E8E9F2E2C3
:1017D000838194818017910719F4148213821082F7
:1017E000BC96CF0185978B5C924290F3E7EDF7E2D0
:1017F000858996898017910711F4118A108A799644
:1018000088E2E930F80708F0AECFF2CFE4E04035E7
:101810005E07B1F5CA010E941B08892B89F110925D
:101820004C04CCE2D0E09CE2D92E26C090E08C9F04
:10183000F0018D9FF00D9C9FF00D1124ED58FD4D92
:1018400085A18823A1F080E594E00E946C09809135
:101850004C048D9DC00111248D589D4D9093722292
:101860008093712282E00E941D3B0E945C0A80915D
:101870004C048F5F80934C0480914C048230B0F212
:10188000F0E2043E1F0749F4C8010E941B08892B9F
:1018900021F00E94420E0E945C0A21E205361207E6
:1018A00049F4C8010E941B08892B21F00E94321CB8
:1018B0000E945C0A81E20D36180749F4C8010E94B3
:1018C0001B08892B21F00E941C1B0E945C0AE1E28C
:1018D00005371E0709F047CFC8010E941B08892B56
:1018E00009F441CF0E94231E3ECF4115510509F452
:1018F0003ACF509372224093712283E00E941D3BA5
:101900000E945C0A80E594E00E941B08892B09F480
:101910002ACF80E594E00E946C0925CF411551053E
:1019200009F421CF50936E2240936D2285E00E94EE
:101930001D3B0E945C0A17CF80915A2290915B2236
:10194000892B09F410CF81E00E941D3B80915A221F
:1019500090915B22892B09F406CF0E94480D03CF9A
:10196000F7011182108283E0DF91CF911F910F91D7
:10197000FF90EF90DF900895CF93DF93EA010E94EC
:10198000A443FC01009741F08091990390919A0340
:10199000968B858BD08FC78BCF01DF91CF91089528
:1019A0000F931F93DF93CF93CDB7DEB760970FB63A
:1019B000F894DEBF0FBECDBF8C01AB018FEF92E07C
:1019C0009A8389831C821B821E821D8218861F8235
:1019D0001A8619861C861B861E861D8680E091E06D
:1019E000988B8F87CE010196B8010E94BC0CFC0138
:1019F000009711F0118B008BCF0160960FB6F89411
:101A0000DEBF0FBECDBFCF91DF911F910F91089523
:101A1000AC0110924E04E8E5F4E020E016C0322F4D
:101A20003F5F80819181892B71F420934E04518313
:101A300040838091990390919A0393838283CA0192
:101A40000E944C3A08953496232F223040F320937D
:101A50004E0408950F931F93CF93DF938A010E9442
:101A6000A939EC01009771F08091990390919A0344
:101A700099A788A71BA70AA785EB91E060E0AE01B4
:101A80000E947907CE01DF91CF911F910F910895A8
:101A9000EF92FF920F931F938091D922863009F025
:101AA0005DC080915A2290915B228050954009F050
:101AB00055C00EE912E010935B2200935A2292E087
:101AC000E92EE092D72286E7F82EF092D8221092E3
:101AD0000C2310920B230E94A1398095909590932E
:101AE0000C2380930B230E945C0A10935B220093CB
:101AF0005A22E092D722F092D82220916F22309180
:101B00007022C901FC01DC01AE59BD4F82E692E0B2
:101B10000D9001920197E1F78FEF92E262E672E099
:101B20000E94A93880915E228093FF2280915F22DB
:101B30008093002380916022809301238091612211
:101B40008093022310920C2310920B230E94A13940
:101B50008095909590930C2380930B230E945C0AB0
:101B60001F910F91FF90EF900895AC011092891989
:101B7000109288191092831920E06BE070E021C068
:101B8000822F90E0869FF001879FF00D969FF00DC9
:101B90001124E45EF64E8285882391F08081918144
:101BA0008417950769F4209383198BE0289FC0015F
:101BB0001124845E964E909389198093881905C0EC
:101BC0002F5F2230E8F22093831980918819909139
:101BD0008919089510928919109288191092831901
:101BE00040E050E020E06BE070E03BE030C0822F4E
:101BF00090E0869FF001879FF00D969FF00D1124D5
:101C0000E45EF64E8285882309F10190F081E02D93
:101C10003097E1F0818D928D009711F0059749F48E
:101C20004115510599F4239FA0011124445E564E9D
:101C30000DC0209383198BE0289FC0011124845E7E
:101C4000964E909389198093881909C02F5F22308E
:101C500070F25093891940938819209383198091C9
:101C60008819909189190895FC0112860190F081DC
:101C7000E02D818D928D059709F414A60895FC013D
:101C8000128E08959F92AF92BF92CF92DF92EF9201
:101C9000FF920F931F93CF93DF9384EE90E20E9405
:101CA0007709109289191092881910928319CBE044
:101CB000D0E00BE02EC0822F90E08C9FF0018D9F32
:101CC000F00D9C9FF00D1124E45EF64E828581306C
:101CD000D9F4209FC0011124845E964E90938919F7
:101CE0008093881902960E945B38892B69F0E091F5
:101CF0008819F091891912860190F081E02D818D6B
:101D0000928D059709F414A6809183198F5F8093B3
:101D1000831920918319223070F210928719109242
:101D20008619109283193EE2A32E35E0B32E22E0ED
:101D3000C22ED12C94E0E92EF12CCBE0D0E08BE048
:101D4000982ED8C090E08A9DD0018B9DB00D9A9DB1
:101D5000B00D1124AC59BB4F9C968C919C9781304F
:101D600009F0C3C0B0938719A093861959968D9135
:101D70009C915A978130910511F18130910538F08D
:101D80008330910559F1049709F0AFC036C09B9696
:101D90008C919B97833018F09C961C92A6C0CD0125
:101DA00083960E945B38892B09F49FC04091861965
:101DB0005091871980E090E060E070E075C0CD013F
:101DC0004B960E945B38892B09F48FC0E0918619ED
:101DD000F0918719D28EC18E13A687C0CD014B9684
:101DE0000E945B38892B09F480C0E0918619F0913C
:101DF0008719F28EE18E13A650C09B968C919B970B
:101E0000833008F444C09B961C929B9710928919CA
:101E1000109288191092831920E020C0822F90E040
:101E20008C9FF0018D9FF00D9C9FF00D1124E45EBE
:101E3000F64E8285882389F0808191818A179B07DD
:101E400061F420938319299DC0011124845E964E6C
:101E5000909389198093881905C02F5F2230F0F282
:101E600020938319E0918819F0918919309749F0EE
:101E700012860190F081E02D818D928D059709F4F5
:101E800014A6E0918619F091871914A62EC0CD01F1
:101E900083960E945B38892B41F1409186195091BD
:101EA000871980E090E0BA010E945B1600918619C4
:101EB000109187196091F9207091FA208091FB2090
:101EC0009091FC2028EE33E040E050E00E947650F4
:101ED000C8018396BA01A9010E949138E091861940
:101EE000F091871983A58F5F83A7809183198F5FF6
:101EF0008093831980918319843008F423CF109242
:101F000085191092841981E080938319CBE1D0E088
:101F10000BE12AC0822F90E08C9FF0018D9FF00D85
:101F20009C9FF00D1124EE5CF64E828D8130B9F449
:101F3000209FF0011124EE5CF64EF0938519E0939A
:101F40008419818D882359F4CF0141960E945B3812
:101F5000892B29F0E0918419F0918519128E8091D6
:101F600083198F5F8093831920918319233090F216
:101F7000DF91CF911F910F91FF90EF90DF90CF9065
:101F8000BF90AF909F900895BF92CF92DF92EF9253
:101F9000FF920F931F93CF93DF93D82EC92EB62EA7
:101FA00079018A01109285191092841981E0809339
:101FB000831921E04BE150E014C0322F3F5F822FA4
:101FC00090E0849FF001859FF00D949FF00D112407
:101FD000EE5CF64E828D882319F4209383190DC090
:101FE000232F233050F320938319233031F40E94A0
:101FF000A33881708F5F80938319909183198BE14F
:10200000989FF0011124EE5CF64EF0938519E09351
:102010008419EF012D2D3C2DC901DC0180E10D90CB
:1020200009928150E1F7B08AE114F104010511052C
:1020300061F0CF014196B801A7010E949138E0916B
:102040008419F0918519118E02C081E0818F8091F1
:10205000831990E02BE130E0829FF001839FF00D27
:10206000929FF00D1124EE5CF64E81E0828F8091FC
:10207000841990918519DF91CF911F910F91FF9055
:10208000EF90DF90CF90BF900895EF92FF920F9363
:102090001F93CF93DF93EC017A018B011092891982
:1020A000109288191092831920E04BE050E014C080
:1020B000322F3F5F822F90E0849FF001859FF00DCB
:1020C000949FF00D1124E45EF64E8285882319F466
:1020D000209383190CC0232F223050F320938319AF
:1020E000223029F40E94A338817080938319E091F3
:1020F00083198BE0E89FF0011124E45EF64EF09323
:102100008919E0938819C193D193CF01B801A70130
:102110000E9491388091831990E02BE030E0829FFB
:10212000F001839FF00D929FF00D1124E45EF64EB6
:1021300081E082878091881990918919DF91CF91F0
:102140001F910F91FF90EF900895EF92FF921F93D0
:10215000CF93DF93EC01109285191092841910929D
:1021600083194BE1E42EF12C24C0812F90E08E9D49
:10217000F0018F9DF00D9E9DF00D1124EE5CF64E4A
:10218000828D882399F0CF01BE0140E150E00E948A
:10219000FB4C009759F48BE1189FC00111248E5C11
:1021A000964E909385198093841907C01F5F1093F2
:1021B0008319109183191330C0F280918419909182
:1021C0008519DF91CF911F91FF90EF900895EF92C5
:1021D000FF921F93CF93DF93EC01109283195BE181
:1021E000E52EF12C1EC0812F90E08E9DF0018F9D79
:1021F000F00D9E9DF00D1124EE5CF64E828D88232D
:1022000069F04089469546954695CF01BE0150E05C
:102210000E94FB4C009711F481E008C01F5F1093EF
:102220008319109183191330F0F280E0DF91CF9180
:102230001F91FF90EF900895CF92DF92EF92FF925F
:102240001F93CF93DF937C01109287191092861908
:10225000109283196EE2C62E65E0D62E1EC0812F25
:1022600090E08C9DE0018D9DD00D9C9DD00D1124A2
:10227000CC59DB4F8CA5882369F0CE01B70140E132
:1022800050E00E94FB4C009729F4D0938719C0932B
:10229000861907C01F5F109383191091831914309A
:1022A000F0F28091861990918719DF91CF911F915B
:1022B000FF90EF90DF90CF900895BF92CF92DF9282
:1022C000EF92FF920F931F93CF93DF93D82EC92ED7
:1022D0008B01B42E790110928719109286191092F1
:1022E000831920E04EE255E014C0322F3F5F822F69
:1022F00090E0849FF001859FF00D949FF00D1124D4
:10230000EC59FB4F84A5882319F4209383190CC042
:10231000232F243050F320938319243029F40E9472
:10232000A3388370809383198091831990E02EE203
:1023300035E0829FF001839FF00D929FF00D1124F4
:10234000EC59FB4FF0938719E0938619EF012D2D7F
:102350003C2DC901DC0180E10D9009928150E1F72B
:10236000CF0140960115110541F0FC01D80188E02C
:102370000D9001928150E1F706C0FC0188E0DF0179
:102380001D928A95E9F7E0918619F0918719B08E30
:10239000F28EE18ECF014B9640E050E060E070E0BD
:1023A0000E9491388091861990918719839640E018
:1023B00050E060E070E00E949138E0918619F09161
:1023C000871913A681E084A7CF01DF91CF911F91D8
:1023D0000F91FF90EF90DF90CF90BF90089520E095
:1023E0004EE255E00DC0822F90E0849FF001859F62
:1023F000F00D949FF00D1124EC59FB4F14A62F5FA4
:10240000243088F320E04BE050E00DC0822F90E0B4
:10241000849FF001859FF00D949FF00D1124E45EE0
:10242000F64E12862F5F223088F320E04BE150E019
:102430000DC0822F90E0849FF001859FF00D949F46
:10244000F00D1124EE5CF64E128E2F5F233088F3D0
:10245000209383198EEF90E890933319809332196B
:1024600010923519109234191092371910923619AA
:10247000109239191092381910923B1910923A198A
:1024800010923D1910923C1910923F1910923E196A
:10249000109241191092401980E48093421981E012
:1024A00080934C1980934B1984EE90E26CE070E0BD
:1024B0000E9482090895DF92EF92FF920F931F937B
:1024C000CF93DF938091DA228F3F09F02CC3809164
:1024D000DB228E3F09F027C38091DC22803809F08F
:1024E00022C38091C520A82FB0E0FD01E550FD4D2D
:1024F0008181882309F017C3A150BD4D8C91882399
:1025000011F08093F020E091C520F0E0E150FD4D06
:1025100064817581868197816115710581059105B9
:1025200061F1E090F120F090F2200091F320109101
:10253000F4200E94853AE616F70608071907E9F025
:10254000E091C520F0E0E150FD4D64817581868108
:1025500097810E94853A6093F1207093F2208093D6
:10256000F3209093F4200E94641B6093F5207093F5
:10257000F6208093F7209093F820E091C520F0E0BA
:10258000E150FD4D608571858285938561157105EA
:102590008105910551F00E94853A6093F92070936E
:1025A000FA208093FB209093FC2010928C191092BB
:1025B0008B1910928E1910928D1940E009C0E42FEA
:1025C000F0E0EE0FFF1FE157F64E118210824F5FD1
:1025D0004330A8F340939D198CE080938A19609151
:1025E0005A2270915B223AC0F901ED52FD4D818172
:1025F000882309F496C28081833071F0853039F0E8
:102600008130E1F4F0938C19E0938B1917C0F093AB
:102610008E19E0938D1912C040E0433079F0542FA9
:102620005F5FE42FF0E0EE0FFF1FE157F64E808171
:102630009181892B09F47CC2452FEFCF80918A19B3
:10264000E091C520F0E0ED52FD4DE80FF11D95A59C
:10265000990F990F990F980F90938A199091C5200F
:1026600080918A19282F30E0290F311D245D3F4FBA
:102670002617370708F4B8CF40939D19E0918D19BC
:10268000F0918E19309771F0648175818681978100
:102690000E94853A6093EC207093ED208093EE20A9
:1026A0009093EF2010929D19DD24D39459C1648139
:1026B0007581868197810E94853A7B018C01E0912A
:1026C0009D19F0E0EE0FFF1FE157F64E0190F081EB
:1026D000E02D60857185828593850E94853AE61696
:1026E000F7060807190708F436C1E0919D19F0E0D4
:1026F000EE0FFF1FE157F64E0190F081E02D80892B
:102700008E3F21F48189803809F425C1838187FFB8
:102710006BC0CF0140960E94A510EC0190939819D0
:1027200080939719E0919D19009789F5F0E0EE0FDD
:10273000FF1FE157F64E0190F081E02D6481758115
:1027400086819781611571058105910509F44CC059
:10275000EF0160966F3F2FEF72072FEF82072FEF89
:10276000920741F012810E94853A9B01AC01CE0193
:10277000612F06C0CE01628120E030E040E050E0F1
:102780000E94C40F90939819809397192DC0F0E080
:10279000EE0FFF1FE157F64E0190F081E02D6481AE
:1027A000758186819781611571058105910549F0D3
:1027B0006F3F2FEF72072FEF82072FEF920739F449
:1027C00004C0CE010E943F0E0FC0D98E0DC00E94E2
:1027D000853AAB01BC01CE0141960E949138E0914F
:1027E0009719F0919819118EE0919D19F0E0EE0F74
:1027F000FF1FE157F64E0190F081E02D838186FFA7
:10280000AAC084819581A681B7810097A105B105F1
:1028100009F4A1C0CF014096628141E050E00E94DE
:10282000B01BDC0190939C1980939B19E0919D193A
:10283000009709F468C0F0E0EE0FFF1FE157F64E75
:102840000190F081E02D64817581868197816F3FD1
:102850002FEF72072FEF82072FEF920709F450C076
:102860000E94853A61527C4180409040F0F4E091B2
:102870009D19F0E0EE0FFF1FE157F64E0190F08139
:10288000E02D64817581868197810E94853A7B0164
:102890008C0180919B1990919C1942960E94353829
:1028A0006E157F0580079107D0F400919B19109158
:1028B0009C190E5E1F4FE0919D19F0E0EE0FFF1F77
:1028C000E157F64E0190F081E02D6481758186819B
:1028D00097810E94853AAB01BC01C80109C0809173
:1028E0009B1990919C19429640E25CE160E070E097
:1028F0000E949138E0919B19F0919C19128E2BC087
:102900005A96DC9228C0F0E0EE0FFF1FE157F64E1A
:102910000190F081E02D6481758186819781EF01BE
:1029200060966F3F2FEF72072FEF82072FEF92070E
:1029300041F012810E94853A9B01AC01CE01612FCA
:1029400006C0CE01628120E030E040E050E001E0CE
:1029500010E00E94781D80919D198F5F80939D19D2
:10296000E0919D19E23058F4F0E0EE0FFF1FE157BF
:10297000F64E0190F081E02D309709F098CE8BED66
:1029800092E20E941C11FC01909396198093951974
:1029900060918B1970918C196115710509F440C013
:1029A000009771F46E5F7F4F8BED92E241E022E081
:1029B00030E00E945D11909396198093951930C074
:1029C000818D928D892B21F482E090E0928F818F0E
:1029D000C0918B19D0918C19229600919519109164
:1029E0009619005F1F4FCE01B80148E050E00E94E9
:1029F000FB4C009779F0D801FE0188E001900D9220
:102A00008150E1F7E0919519F091961982E090E0FC
:102A1000928F818FE0919519F091961981E0808FC6
:102A2000E091C520F0E0E150FD4D82819381E0917D
:102A30009519F0919619892B09F442C0309771F4D9
:102A40008BED92E260E070E041E025E030E00E9432
:102A50005D11909396198093951902C081E0808F43
:102A600080919519909196190E94B50D8C019093C3
:102A70009A1980939919E091C520009791F40091DB
:102A8000951910919619F0E0E150FD4D82819381E6
:102A90000E94813AAC0160E070E0C8010E944510DC
:102AA0001CC0F0E0E150FD4D828193810E94813A8B
:102AB000AC0160E070E0C80102960E9491380DC040
:102AC000309759F0CF010E94B50D90939A198093D9
:102AD0009919009711F00E94340EE0919519F09128
:102AE0009619309701F1E35DFA4FA081ED52F54060
:102AF000AA23C9F0A0935A2210925B2223ED32E25E
:102B0000AF01435D5F4FC901BA014A2F50E00E94F7
:102B1000084DE0919519F0919619E35DFA4F1082F6
:102B20000CC040939D1910925B2210925A2205C04E
:102B30002D523D4D3183208381CDDF91CF911F9167
:102B40000F91FF90EF90DF900895CF93DF9383ED87
:102B500092E220E62093D3221092D4221092D62221
:102B60001092D5222AE32093D9222FEF2093DA2244
:102B7000FC0178962FEF32E03093EC222093EB2289
:102B80001382128215821482178216821186108691
:102B9000138612861586148620E032E03787268752
:102BA0000896BF010E94B41A4091C520242F30E03E
:102BB000F901E550FD4D85E880831182F901E1506E
:102BC000FD4D10821182128213821092D7228091C1
:102BD000DB229091DC22892BA1F58091DD2290915E
:102BE000DE22892B71F58091DF229091E022892BE2
:102BF00041F58091E1229091E222892B11F580919B
:102C0000E3229091E422892BE1F48091E5229091D6
:102C1000E622892BB1F48091E7229091E822892B5A
:102C200081F48091E9229091EA22892B51F488E085
:102C30008093D822205D3F4F30935B2220935A220D
:102C400029C0842F90E0805C9F4F90935B228093FB
:102C50005A2288E18093D822F901ED5FFC4DF09370
:102C60008C19E0938B1981E0808382E08183329616
:102C7000A2E6B2E288E00D9001928150E1F78091E6
:102C80008B1990918C190A96FC0186E0DF011D9248
:102C90008A95E9F78091C520C82FD0E0C550DD4D59
:102CA0001B821A820E949D39809590959B838A830E
:102CB000DF91CF9108950F931F93CF93DF938C01F2
:102CC000EA011092C52080E68093D3221092D4228C
:102CD0001092D6221092D5228AE38093D9229FEFB8
:102CE0009093DA22EBEEF2E261157105B9F490935C
:102CF000EB2282E081831382128215821482178272
:102D0000168211861086128681E0838794878D85CE
:102D100085878E859F859787868707C0DF01FB01A2
:102D200080E101900D928150E1F787E88093FB22CA
:102D30001092FC221092FF22109200231092012385
:102D400010920223A3E0B3E2FE0180E101900D9214
:102D50008150E1F71092D722CE0160E840E050E0C8
:102D60000E94B01B892BE1F50115110549F0ABED6F
:102D7000B2E2F80180E101900D928150E1F706C0C6
:102D80008BED92E26BEE72E20E94B41A88E28093BD
:102D9000D82280E590E090935B2280935A22E091C4
:102DA000C520F0E0ED5EFC4DF0938C19E0938B199B
:102DB00081E0808382E081833296A2E6B2E288E0FD
:102DC0000D9001928150E1F780918B1990918C19AF
:102DD0000A96FC0186E0DF011D928A95E9F729C079
:102DE0001092DC221092DB221092DE221092DD2261
:102DF0001092E0221092DF221092E2221092E12241
:102E00001092E4221092E3221092E6221092E52220
:102E10001092E8221092E7221092EA221092E92200
:102E200088E18093D82280E490E090935B228093A5
:102E30005A228091C520C82FD0E0C550DD4D1B829D
:102E40001A820E949D39809590959B838A83DF9199
:102E5000CF911F910F910895DF92EF92FF920F9300
:102E60001F93CF93DF939091C520E92FF0E0DF010E
:102E7000A150BD4DFC908091DA228F3F09F041C1F5
:102E8000E550FD4D8181882309F03BC114968C915A
:102E900014978F3F09F435C120E4D22EDF20F6FECF
:102EA00005C08091EB228F3F09F42BC184E1809310
:102EB0008A1910928C1910928B19C0915A22D091B4
:102EC0005B2240E050E064E1292F30E0245D3F4F79
:102ED0000FC0FC01ED52FD4D9181992309F40BC106
:102EE0008081823009F4AF01990F990F990F690F12
:102EF000C901860F911D8C179D0758F350938C19AB
:102F000040938B1960938A19CD01049660E840E0E4
:102F100050E00E94B01BFC0190939C1980939B1978
:102F2000009769F080899189892B09F0EAC0809126
:102F3000C52090E08D5F9C4D0E94111CE2C08091E5
:102F4000C52090E08D5F9C4D0E941C118C019093D8
:102F5000961980939519009709F4D3C0C0918B19E5
:102F6000D0918C19209711F420E00AC0BC01605F59
:102F70007F4FCE01029648E050E00E94FB4C282F84
:102F800080E8E82EEF20F801818D928D009781F581
:102F9000209709F4B6C0D8015096FE01329688E019
:102FA00001900D928150E1F7C0919519D091961939
:102FB000DD20C9F081E090E09A8F898F6091F52043
:102FC0007091F6208091F7209091F82028EE33E060
:102FD00040E050E00E947650CE014B96BA01A90124
:102FE0000E94913861C082E090E09A8F898F5CC026
:102FF000F5FC0BC0222349F0019709F082C082E062
:1030000090E0F801928F818F7CC0209749F0D80121
:103010005096FE01329688E001900D928150E1F7C2
:10302000DD20F1F0009195191091961981E090E062
:10303000F801928F818F6091F5207091F620809138
:10304000F7209091F82028EE33E040E050E00E9415
:103050007650C8014B96BA01A9010E94913810C060
:1030600080918B1990918C19892B51F0222341F07A
:10307000E0919519F091961982E090E0928F818FFE
:10308000E0919519F0919619808D882369F0EE20D2
:1030900059F4CF010E94B50D90939A198093991914
:1030A000009711F00E94340EE0919519F091961955
:1030B000E08EE0919519F0919619E35DFA4FA081A9
:1030C000ED52F540AA23E9F0A0935A2210925B2218
:1030D00023ED32E2AF01435D5F4FC901BA014A2FD0
:1030E00050E00E94084DE0919519F0919619E35D2A
:1030F000FA4F10820AC050938C1940938B19609339
:103100008A1910925B2210925A22DF91CF911F915F
:103110000F91FF90EF90DF900895EF92FF920F9341
:103120001F93CF93DF938091DA228F3F09F0F2C192
:103130008091C520482F50E0FA01E150FD4D848177
:103140008F3F09F4E7C1FA01E550FD4D81818823E5
:1031500009F0E0C110928C1910928B1984E18093D0
:103160008A19C0915A22D0915B2220E030E064E1BC
:10317000FA01BC9611C0DC01AD52BD4D11969C9177
:103180001197992309F4C0C18C91813009F49D01F4
:10319000990F990F990F690FCF01860F911D8C1709
:1031A0009D0748F320938B1930938C1960938A19EB
:1031B000232B09F472C08091DB229091DC22892BB1
:1031C00059F58091DD229091DE22892B29F580919D
:1031D000DF229091E022892BF9F48091E1229091F5
:1031E000E222892BC9F48091E3229091E422892B79
:1031F00099F48091E5229091E622892B69F48091DF
:10320000E7229091E822892B39F48091E92290916C
:10321000EA22892B09F47EC18BED92E20E941C11F7
:10322000EC01909396198093951960918B19709188
:103230008C19009751F46E5F7F4F8BED92E240E066
:1032400022E030E00E945D1128C032E0E32EF12C34
:10325000E60EF71E8C01005F1F4FC701B80148E062
:1032600050E00E94FB4C009781F0D801F70188E004
:1032700001900D928150E1F7E0919519F091961926
:1032800082E090E0928F818F08C0898D9A8D892B82
:1032900021F482E090E09A8F898F8091C52090E0A0
:1032A0008D5F9C4D60E840E050E00E94B01B909321
:1032B0009C1980939B19892B09F42CC18091DB22E6
:1032C0009091DC22892B09F074C08091DD229091CD
:1032D000DE22892B09F06DC08091DF229091E022DF
:1032E000892B09F066C08091E1229091E222892B1E
:1032F00009F05FC08091E3229091E422892B09F0CC
:1033000058C08091E5229091E622892B09F051C0A6
:103310008091E7229091E822892B09F04AC08091A0
:10332000E9229091EA22892B09F043C08BEE92E2C8
:103330000E94051C882309F4EDC0E0919B19F091CF
:103340009C1980899189892B61F18FEF92E090938C
:10335000EC228093EB221092EE221092ED2210923A
:10336000F0221092EF221092F2221092F12210928B
:10337000F4221092F3221092F6221092F52210926B
:10338000F8221092F72280E091E09093FA22809345
:10339000F9228BED92E26BEE72E20E94B41A90E297
:1033A00055C08091C52090E08D5F9C4D0E94111CFE
:1033B000B1C08BED92E260E840E050E00E94B01BAB
:1033C000892B09F0A7C08BEE92E20E94051C88238E
:1033D000B9F0EBEEF2E2DF01509780E10D9001923F
:1033E0008150E1F78091C520E82FF0E0ABEDB2E22B
:1033F000ED5FFC4D80E101900D928150E1F725C019
:103400008BEE92E260E840E050E00E94B01B209119
:103410009B1930919C192817390709F07BC0EBEEF6
:10342000F2E2DF01509780E10D9001928150E1F7C7
:103430008091C520E82FF0E0ABEDB2E2ED5FFC4DEE
:1034400080E101900D928150E1F790E61092C52045
:1034500080E68093D3221092D4221092D62210922A
:10346000D5221092D72288E28093D8228AE38093D3
:10347000D9228FEF8093DA2288E88093FB22109282
:10348000FC229093FF22A3E0B3E220919B1930919C
:103490009C19C901FC0180E101900D928150E1F776
:1034A00080E590E090935B2280935A22E091C520C2
:1034B000F0E0ED5EFC4DF0938C19E0938B1982E007
:1034C000808381833296A2E6B2E288E00D90019279
:1034D0008150E1F780918B1990918C190A96FC012B
:1034E00086E0DF011D928A95E9F78091C520C82FFB
:1034F000D0E0C550DD4D1B821A820E949D39809517
:1035000090959B838A830AC030938C1920938B19E2
:1035100060938A1910925B2210925A22DF91CF9108
:103520001F910F91FF90EF90089540E020E030E070
:10353000FC01E20FF31F5081FB01E20FF31FE0815A
:103540005E1731F4485F2F5F3F4F403889F70AC05C
:10355000E527842F885FE7FD05C04F5F481711F00E
:10356000EE0FF9CF842F0895EF92FF920F931F93E0
:10357000CF93DF93F82EE92EEB0188818E3F21F463
:103580008981803819F43BC08F3FC9F130E020E0D9
:1035900061E00DE110E02EC0862F90E0809FA00139
:1035A000819F500D909F500D1124FA01E451FF4D61
:1035B00082A193A10197E9F4DE01FA01E250FF4DE7
:1035C00080E04C919081491731F4885F11963196D3
:1035D0008038B9F70AC09427482F485F97FD05C087
:1035E0008F5F841711F0990FF9CF831710F0382FE0
:1035F000262F6F5F633080F26093A21901C020E034
:1036000030E08DE190E0289FF001299FF00D389F78
:10361000F00D11242F2D3E2DC901DC01E250FF4D8C
:1036200080E101900D928150E1F7DF91CF911F91E0
:103630000F91FF90EF9008950E94EA0D892B91F46D
:103640008091A119833070F40E94A5158091A11971
:103650008F5F8093A1198DE691E264EF71E00E9483
:10366000820908958DE691E20E9480081092A119C6
:1036700008958091A119882359F40E94A3386DE719
:1036800070E00E944F50BC018DE691E20E948209D9
:103690000895FC0180899189892BA9F480919E1954
:1036A00090919F19892B79F4F0939F19E0939E19BB
:1036B0000E94A3386DE770E00E944F50BC0185E680
:1036C00091E20E94820908958F929F92AF92BF92D9
:1036D000DF92EF92FF920F931F936091F120709110
:1036E000F2208091F3209091F4200E942C4A20E057
:1036F00030E040E05FE30E944E480E9478464B0174
:103700005C010E94A338D82E0E94A338FD2CEE2421
:10371000E80EF91E00E010E06091F1207091F220B7
:103720008091F3209091F4200E942C4A0E947846C8
:103730009B01AC01C801B7010E9476509B01AC010E
:10374000280D391D4A1D5B1DB901CA011F910F913A
:10375000FF90EF90DF90BF90AF909F908F90089573
:10376000CF92DF92EF92FF920F931F93CF93DF934D
:103770007C01062FEA011092A2190695069506957E
:103780008DE1C82ED12C31C0212F30E02C9DF001CD
:103790002D9DF00D3C9DF00D1124E451FF4D82A1B3
:1037A00093A18F5F9F4FF1F085A596A58C179D077C
:1037B00011F02097B9F42C9DC0012D9D900D3C9DDA
:1037C000900D112482509F4DB701402F50E00E9470
:1037D000FB4C009739F48DE1189F90011124225081
:1037E0003F4D09C01F5F1093A2191091A219133009
:1037F00058F220E030E0C901DF91CF911F910F9185
:10380000FF90EF90DF90CF90089565E571E240E181
:1038100050E00E94FB4C9C0180E0232B09F481E0E6
:103820000895BC0180919E1990919F1940E150E04C
:103830000E94FB4C009791F485E691E20E9480087B
:10384000E0919E19F0919F198FEF9FEF918B808BE4
:1038500010929F1910929E191092A0198FEF9FEF4E
:103860000E94EA5040919E1950919F1941155105AF
:1038700009F468C09091A0198091FD20981748F52F
:1038800080E090E060E070E00E945B168091A019FB
:103890008F5F8093A0196091F9207091FA20809138
:1038A000FB209091FC2028EE33E040E050E00E94A5
:1038B0007650CA01B9012DE730E040E050E00E94A7
:1038C00030509B01AC0185E691E2B9010E9482096A
:1038D000089585E691E20E948008E0919E19F0919A
:1038E0009F1981E090E0918B808B10929F1910922C
:1038F0009E191092A0191092A21920E04DE150E0FB
:103900001DC0322F3F5F822F90E0849FF001859F82
:10391000F00D949FF00D1124E451FF4D82A193A16D
:10392000892B59F42093A2198DE1289FC0011124FD
:1039300082509F4D0E94491B0895232F233008F386
:103940002093A2190895CF93DF93DC01EC01289610
:10395000FB0188E0019009928150E1F718968C9163
:10396000189792E0892718968C93DF91CF9108954C
:1039700080E095E0A0E0B0E08093EC209093ED2013
:10398000A093EE20B093EF2080E48093F02080E3BA
:1039900095E7A0E0B0E08093F1209093F220A0930F
:1039A000F320B093F4200E94641B6093F520709381
:1039B000F6208093F7209093F82088EE93E0A0E023
:1039C000B0E08093F9209093FA20A093FB20B0936D
:1039D000FC2081E08093FD208EEF90E89093FF2003
:1039E0008093FE2010920121109200211092032159
:1039F00010920221109205211092042110920721A9
:103A000010920621109209211092082110920B2188
:103A100010920A2110920D2110920C21A6E0B1E221
:103A2000E2E6F2E288E001900D928150E1F78091A8
:103A3000062192E089278093062110920F2110928F
:103A40000E2183E090E090931A218093192181E068
:103A50008093182121E06DE170E04FEF5FEF0EC021
:103A6000822F90E0869FF001879FF00D969FF00DCA
:103A70001124E451FF4D53A342A32F5F233080F361
:103A80002093A2199FEF9093552182E080935621B5
:103A900010925721109258211092592110925A21B8
:103AA00010925B2110925C2110925D2110925E2198
:103AB00010925F2181E08093602190936121809139
:103AC0006722809362218091682280936321809194
:103AD0006922809364218EEF90E20E94491B0E942C
:103AE000391B85E791E26DE770E00E948209089535
:103AF000AF92BF92CF92DF92EF92FF920F931F93FC
:103B0000CF93DF93B82EA92E69017A0101301105F8
:103B100019F4603409F08CC01092A21920E06DE114
:103B200070E081C0422F50E0322F3F5F469FD001AE
:103B3000479FB00D569FB00D1124FD01E451FF4D7C
:103B400082A193A18F5F9F4F09F06CC02093A219AF
:103B5000FD01E250FF4D8B2D9A2D9C01D90180E192
:103B60000D9001928150E1F70130110509F58DE1C9
:103B700090E0489FF001499FF00D589FF00D1124EF
:103B8000EA5FFE4DA2E6B2E288E00D90019281501C
:103B9000E1F78DE190E0489FF001499FF00D589FBB
:103BA000F00D1124E451FF4D828D92E08927828F20
:103BB0008091A21990E0CDE1D0E08C9F90018D9F83
:103BC000300D9C9F300D1124F901E451FF4D13A2DB
:103BD00012A216A705A7C114D104E104F104A9F0AB
:103BE000C901805F9E4DB701A6010E949138809166
:103BF000A21990E08C9FF0018D9FF00D9C9FF00D1D
:103C00001124E451FF4D14A602C081E084A78091E5
:103C1000A2192DE1829FC001112482509F4D0E9464
:103C2000491B06C0232F233008F47CCF2093A21910
:103C3000DF91CF911F910F91FF90EF90DF90CF9088
:103C4000BF90AF9008950F931F93CF93DF9381E0C0
:103C50008093A219CDE1D0E00FEF1FEF2DC090E0CF
:103C60008C9F90018D9F300D9C9F300D1124F90188
:103C7000E451FF4D82A193A18F5F9F4FC1F084A5B6
:103C80008130A9F0C901805F9E4D0E945B38892B6D
:103C900071F08091A21990E08C9FF0018D9FF00D42
:103CA0009C9FF00D1124E250FF4D118B008B8091F1
:103CB000A2198F5F8093A2198091A219833078F2A4
:103CC00085E791E20E947709DF91CF911F910F91D3
:103CD0000895FC019093A4198093A3190084F185A1
:103CE000E02D8DEA93E209958FE99EE10E94970904
:103CF00091E09093B61E1092B71E8EEF8093B81E7F
:103D000080E88093B91E9093C01E9093C11E8AEAEA
:103D10008093C21E8093C31E82E08093CE1E0895BE
:103D2000BC0185E10E946236E091A319F091A419CB
:103D3000309721F00480F581E02D09950895EF92E8
:103D4000FF920F931F93DF93CF93CDB7DEB72897E2
:103D50000FB6F894DEBF0FBECDBF8C011092A9192B
:103D60001092A7190E9490360E94FF359093A619D1
:103D70008093A5198091D922863029F483E062E0EE
:103D800070E00E9443367E010894E11CF11C01158D
:103D9000110521F4C7016EEE71E002C0C701B80140
:103DA0000E949937E091A519F091A6193396F093E6
:103DB000CD1EE093CC1E33978091A719E80FF11D1B
:103DC000128211828091A719E091A519F091A6198C
:103DD000E80FF11D83E080838091D422282F30E00A
:103DE000C9018F709070892B09F03FC08091D52256
:103DF0009091D622892BC9F58091A719E091A51938
:103E0000F091A619E80FF11D818180648183809172
:103E1000D322282F30E0C9018F709070892B81F454
:103E20008091D422807F61F48091A719E091A51937
:103E3000F091A619E80FF11D8181806881835FC030
:103E4000E091CC1EF091CD1E44E0220F331F4A9525
:103E5000E1F78091D42282958F70822B80838091AC
:103E6000CC1E9091CD1E019646C08091D32290E049
:103E70008F709070892B51F5822F807F39F580915A
:103E8000A719E091A519F091A619E80FF11D8181FC
:103E900080688183E091CC1EF091CD1E9091D42258
:103EA0009F708091D322807F982B9083E091CC1ECD
:103EB000F091CD1E8091D5229091D622928381835C
:103EC0008091CC1E9091CD1E039615C0E091CC1E22
:103ED000F091CD1E8091D3229091D422A091D52231
:103EE000B091D62280839183A283B3838091CC1E2C
:103EF0009091CD1E04969093CD1E8093CC1E809100
:103F0000D922813161F48091A719E091A519F0912E
:103F1000A619E80FF11D8181806281830EC0E091B6
:103F2000CC1EF091CD1E80838091CC1E9091CD1E31
:103F300001969093CD1E8093CC1E8091DA2280341E
:103F400079F08F3FC9F0813011F58091A719E09188
:103F5000A519F091A619E80FF11D818188600AC0AA
:103F60008091A719E091A519F091A619E80FF11D0C
:103F700081818061818319C08091A719E091A51981
:103F8000F091A619E80FF11D81818861F3CFE091CE
:103F9000CC1EF091CD1E80838091CC1E9091CD1EC1
:103FA00001969093CD1E8093CC1E1092CE1E31C0F0
:103FB000812F90E0FC0133E0EE0FFF1F3A95E1F70F
:103FC000880F991FE80FF91FEA54F14E8081813064
:103FD000E9F4212F30E0C90103E0880F991F0A9509
:103FE000E1F7220F331F820F931F8854914E6BED20
:103FF00072E248E050E00E94FB4C009739F48AE0FE
:10400000189FD0011124AA54B14E09C01F5F10930C
:10401000CE1E1091CE1E123058F2A0E0B0E0B09348
:10402000CB1EA093CA1E109709F49CC08091A719BB
:10403000E091A519F091A619E80FF11D11968C9148
:104040008295807F9281892B82838091622292E087
:1040500089279091E3229817B1F59091E4228091FD
:104060006322981781F59091E52280916422981738
:1040700051F59091E62280916522981721F5909153
:10408000E722809166229817F1F49091E8228091BE
:1040900067229817C1F49091E922809168229817BD
:1040A00091F49091EA2280916922981761F48091AD
:1040B000A719E091A519F091A619E80FF11D8281C9
:1040C000806C828365C08091E3229091E422892BE9
:1040D00059F58091E5229091E622892B29F580916E
:1040E000E7229091E822892BF9F48091E92287FD5B
:1040F0001BC08091A719E091A519F091A619E80FAE
:10410000F11D828180688283E091CC1EF091CD1EEA
:104110008091E9229091EA22918380838091CC1E44
:104120009091CD1E029630C08091A719E091A519FB
:10413000F091A619E80FF11D82818064828320919D
:10414000CC1E3091CD1EC901DC01E3EEF2E288E025
:1041500001900D928150E1F78091CC1E9091CD1E7F
:10416000089612C08091CC1E9091CD1E9C01D90161
:10417000EBEDF2E280E101900D928150E1F7809148
:10418000CC1E9091CD1E40969093CD1E8093CC1E58
:104190008091EB228F3F09F065C08091ED229091D4
:1041A000EE22892B09F050C08091EF229091F022ED
:1041B000892B09F049C08091F1229091F222892B3C
:1041C00009F042C08091F3229091F422892BE1F50D
:1041D0008091F5229091F622892BB1F58091F722FA
:1041E0009091F822892B81F58091F922882361F53D
:1041F0008091FA228150823038F58091A719E091A0
:10420000A519F091A619E80FF11D828188608283BB
:10421000E091CC1EF091CD1E80EA8083E091CC1E0F
:10422000F091CD1E8091EC2290E08F709070880FFD
:10423000991F2081282B2083E091CC1EF091CD1E68
:104240008091FA228183BFC08091CC1E9091CD1EB7
:104250009C01D901EBEEF2E280E101900D928150D8
:10426000E1F7E2C01092CE1E31C0812F90E0FC0138
:1042700073E0EE0FFF1F7A95E1F7880F991FE80FA3
:10428000F91FEA54F14E80818130E9F4212F30E0AA
:10429000C90153E0880F991F5A95E1F7220F331F88
:1042A000820F931F8854914E6BEE72E248E050E00B
:1042B0000E94FB4C009739F48AE0189FD00111242A
:1042C000AA54B14E09C01F5F1093CE1E1091CE1E8E
:1042D000123058F2A0E0B0E0B093CB1EA093CA1EFB
:1042E000109709F494C08091A719E091A519F09155
:1042F000A619E80FF11D828111969C91892B82836A
:10430000FE013196898192E089279091F3229817D6
:1043100079F59091F4228181981751F59091F522C9
:104320008281981729F59091F6228381981701F5DB
:104330009091F72284819817D9F49091F822858181
:104340009817B1F49091F9228681981789F4909189
:10435000FA228781981761F48091A719E091A51935
:10436000F091A619E80FF11D82818C60828365C0EF
:104370008091F3229091F422892B59F58091F522B6
:104380009091F622892B29F58091F7229091F822BD
:10439000892BF9F48091F92287FD1BC08091A71920
:1043A000E091A519F091A619E80FF11D82818860AE
:1043B0008283E091CC1EF091CD1E8091F9229091E4
:1043C000FA22918380838091CC1E9091CD1E02961B
:1043D00030C08091A719E091A519F091A619E80FB6
:1043E000F11D8281846082832091CC1E3091CD1E8C
:1043F000C901DC01E3EFF2E288E001900D92815007
:10440000E1F78091CC1E9091CD1E089612C080914C
:10441000CC1E9091CD1E9C01D901EBEEF2E280E121
:1044200001900D928150E1F78091CC1E9091CD1EAC
:1044300040969093CD1E8093CC1E88E28093A9195C
:104440008091D922813109F064C09091FB22809142
:10445000FC22805B904F0F9770F59091FD22809128
:10446000FE2220EF803B920730F18F5B904F18F5D2
:10447000E091CC1EF091CD1E8BEF8083E091CC1E9D
:10448000F091CD1E9091FE22905B8091FC2282954E
:10449000807F980F9183E091CC1EF091CD1E80918A
:1044A000012390910223938382838091CC1E90916B
:1044B000CD1E049625C0E091CC1EF091CD1E88EF54
:1044C0008083E091CC1EF091CD1E8091FB229091D3
:1044D000FC22A091FD22B091FE2281839283A383CE
:1044E000B483E091CC1EF091CD1E80910123909178
:1044F0000223968385838091CC1E9091CD1E0796D2
:104500009093CD1E8093CC1E8091A919885F8093D3
:10451000A919A091CC1E8091A519A81BA093A71939
:104520008091A919482F50E0E0915A22F0915B2226
:10453000E41BF50B2A2F30E086E690E0821B930BFC
:104540007E010894E11CF11C6091A5197091A619D7
:104550008E179F0708F0D9C0CB0104964A2F50E070
:104560000E94114DE091A519F091A61980915A224F
:1045700090915B22906C9083E091A519F091A6191F
:1045800080915A228183E091A519F091A61980911A
:10459000AF1E8283E091A519F091A6198091AE1EFD
:1045A00083838091A7198C5F8093A71916E6412F0A
:1045B000481B487F4093A8196091A5197091A619CE
:1045C000680F711D2091A91930E02D523D4DCB018E
:1045D000B90150E00E94084D2091A7198091A819B7
:1045E00090E0820F911D0E94FA35C7010E94901E33
:1045F0002091A9198091A81990E0820F911D9093A4
:10460000AD1E8093AC1E85E08093A719E091A5199B
:10461000F091A61980915A2290915B22906E90831E
:10462000E091A519F091A61980915A228183809179
:10463000A719181B187F1093A81987014CC0E09187
:10464000A519F091A61983E0369527958A95E1F78B
:10465000248360915A2270915B224091AC1E50914C
:10466000AD1E9B01241B350B8091A81990E02817E3
:10467000390720F4862F841B8093A8198091A719ED
:104680006091A5197091A619680F711D4091A81924
:104690002091AC1E3091AD1E2D523D4DCB01B90184
:1046A00050E00E94084D2091A7198091A81990E030
:1046B000820F911D0E94FA35C8010E94901E209120
:1046C000A8198091AC1E9091AD1E820F911D909300
:1046D000AD1E8093AC1E2091AC1E3091AD1E80911A
:1046E0005A2290915B222817390708F4A8CF8091AD
:1046F000AE1E9091AF1E01969093AF1E8093AE1E9A
:104700001092AD1E1092AC1E1AC0260F371F4D52CC
:104710005D4DC901BA01AF010E94084D2091A71952
:1047200080915A2290915B22820F911D2091A919AC
:10473000821B91090E94FA35C7010E94901E81E0F8
:1047400028960FB6F894DEBF0FBECDBFCF91DF9194
:104750001F910F91FF90EF9008951F93CF93DF93D8
:104760001092A9191092A7190E94FF359093A619CB
:104770008093A51982EB9EE10E94F337892B41F0CB
:104780001092AB1E1092AA1E1092AD1E1092AC1E7B
:10479000E091A519F091A619908180E02181422F26
:1047A00050E0482B592BCA018070987F892F992798
:1047B000803C910549F0803E9105A9F0C0E0D0E031
:1047C00010E020E030E01DC0EA01D770928180E067
:1047D000238130E0282B392B8091A7198C5F80939F
:1047E000A71910E00EC01481928180E0238130E08F
:1047F000282B392BEA01D7708091A7198B5F809302
:10480000A7198091AC1E9091AD1E892BF1F02097D5
:1048100009F4E7C38091AA1E9091AB1EC817D9076F
:1048200009F0DFC38091B01E9091B11E82179307EB
:1048300009F0D7C384E10E945736BC018DE791E2AD
:104840000E94AA37892BC9F4CCC32097B1F0D0932A
:10485000AB1EC093AA1E3093B11E2093B01E82EBF4
:104860009EE161E772E00E94153884E10E945736AC
:10487000BC018DE791E20E9499375091A7195530FC
:1048800009F43DC32091A5193091A619852F90E018
:10489000D901A80FB91F4C91433021F0413409F0E0
:1048A000A0C315C3FC013396E20FF31FF093CD1E96
:1048B000E093CC1E11968C9186FD22C087FD0DC021
:1048C00081919191A191B1918093AA199093AB1983
:1048D000A093AC19B093AD190EC080E68093AA19CD
:1048E00080818F708093AB19818192819093AD19F3
:1048F0008093AC193396F093CD1EE093CC1E1BC071
:1049000087FD10C0808182958F7080668093AA1980
:1049100081918295807F8093AB19F093CD1EE093B7
:10492000CC1E05C080E68093AA191092AB19109294
:10493000AD191092AC19A091A519B091A61980914A
:10494000A719FD01E80FF11D818185FD0BC0E091E4
:10495000CC1EF091CD1E81918093B019F093CD1EA5
:10496000E093CC1E8091A719FD01E80FF11D818114
:1049700090E0887190708830910561F089309105E0
:104980001CF4892B79F019C08031910529F04897E2
:10499000A1F406C081E001C080E48093B1190DC08C
:1049A0008FEFFBCFE091CC1EF091CD1E81918093D3
:1049B000B119F093CD1EE093CC1E8091A719FD0193
:1049C000E80FF11D828190E08073907064E095950E
:1049D00087956A95E1F7382F1092CE1E20E02CC003
:1049E000822F90E0FC0153E0EE0FFF1F5A95E1F794
:1049F000880F991FE80FF91FEA54F14E808181302A
:104A0000D1F4822F90E0FC0173E0EE0FFF1F7A9546
:104A1000E1F7880F991FE80FF91FEA54F14E8181E1
:104A2000831749F42093CE1E8AE0289FA001112409
:104A30004A54514E07C02F5F223090F22093CE1E71
:104A400040E050E05093CB1E4093CA1E8091A719BE
:104A5000A80FB11D12968C91282F30E0207C307069
:104A60002034310509F471C02134310524F4232B9D
:104A700009F48BC0A0C020383105D1F0203C3105AD
:104A800009F099C04115510509F439C2A2EBB9E109
:104A9000FA01329688E001900D928150E1F784E1AD
:104AA0000E945736BC0182EB99E10E94A31C83C08F
:104AB000A091CC1EB091CD1E8C9187FD23C04115D5
:104AC000510509F41CC2A2EBB9E1FA01329688E063
:104AD00001900D928150E1F786E0EAEBF9E1DF0108
:104AE0001D928A95E9F7E091CC1EF091CD1E81913F
:104AF00091919093C1198093C019F093CD1EE093CA
:104B0000CC1E59C080FDFBC111968C91119781502C
:104B1000823008F0F4C18FEF8093B2198C918695A2
:104B20008F708093B3198DE024EB39E1F901119274
:104B30008A95E9F711968C9111978093C119129675
:104B4000B093CD1EA093CC1E36C04115510509F47B
:104B5000D6C1A2EBB9E1FA01329688E001900D923C
:104B60008150E1F7AAEBB9E18091CC1E9091CD1E66
:104B70009C01F90188E001900D928150E1F780914C
:104B8000CC1E9091CD1E089612C0A2EBB9E1809187
:104B9000CC1E9091CD1E9C01F90180E101900D92F7
:104BA0008150E1F78091CC1E9091CD1E409690935C
:104BB000CD1E8093CC1EA091A519B091A61980910D
:104BC000A719FD01E80FF11D328133701092CE1E3E
:104BD00020E02CC0822F90E0FC0153E0EE0FFF1F7D
:104BE0005A95E1F7880F991FE80FF91FEA54F14E23
:104BF00080818130D1F4822F90E0FC0173E0EE0FD0
:104C0000FF1F7A95E1F7880F991FE80FF91FEA5403
:104C1000F14E8181831749F42093CE1E8AE0289FAC
:104C2000A00111244A54514E07C02F5F223090F248
:104C30002093CE1E40E050E05093CB1E4093CA1EFE
:104C40008091A719A80FB11D12968C91282F30E0E2
:104C50002C7030702430310509F471C025303105D5
:104C600024F4232B09F48BC0A0C028303105D1F0E7
:104C70002C30310509F099C04115510509F43FC1A7
:104C8000A2ECB9E1FA01329688E001900D928150D0
:104C9000E1F785E10E945736BC0182EC99E10E9460
:104CA000A31C83C0A091CC1EB091CD1E8C9187FD1A
:104CB00023C04115510509F422C1A2ECB9E1FA0162
:104CC000329688E001900D928150E1F786E0EAEC9F
:104CD000F9E1DF011D928A95E9F7E091CC1EF09190
:104CE000CD1E819191919093D1198093D019F09319
:104CF000CD1EE093CC1E59C080FD01C111968C9150
:104D000011978150823008F0FAC08FEF8093C2195A
:104D10008C9186958F708093C3198DE024EC39E1D6
:104D2000F90111928A95E9F711968C911197809368
:104D3000D1191296B093CD1EA093CC1E36C041154A
:104D4000510509F4DCC0A2ECB9E1FA01329688E021
:104D500001900D928150E1F7AAECB9E18091CC1E4F
:104D60009091CD1E9C01F90188E001900D92815037
:104D7000E1F78091CC1E9091CD1E089612C0A2EC56
:104D8000B9E18091CC1E9091CD1E9C01F90180E18A
:104D900001900D928150E1F78091CC1E9091CD1E33
:104DA00040969093CD1E8093CC1E8091A919885D6A
:104DB0008093A9198091A719E091A519F091A619DE
:104DC000E80FF11D818185FF56C0A091CC1EB091E6
:104DD000CD1E8C918C7F883F09F04DC081E180937E
:104DE000B0198C91883F29F18B3F09F088C0EAEA1D
:104DF000F9E1B89611968C91119782958F7090E099
:104E000080559F409093D219818311968C91119770
:104E100090E08F70907080559F40928383831296AC
:104E20008D919C9113979093D9198093D8191496CA
:104E300019C011968D919C9112979093D3198093DC
:104E4000D21913968D919C9114979093D5198093B4
:104E5000D41915968D919C9116979093D91980939A
:104E6000D8191796B093CD1EA093CC1E8091A91986
:104E7000885F8093A9198091CC1E9091A519891BF8
:104E80008093A719209771F41092AE190E942D36C5
:104E90009091A91998522091A719921B980F90935D
:104EA000AF1908C0A897D093AE19A8969E012852B2
:104EB0002093AF198091B019813109F58091AE1915
:104EC0009091AF199093D7198093D61918C0852F58
:104ED0008F5F8093A719AAEAB9E1F901E80FF11DE4
:104EE00088E201900D928150E1F78091A719885DC9
:104EF0008093A7198091A919885D8093A9190E94B0
:104F00002D369091A719482F491B4093A819212F9E
:104F100030E053E0220F331F5A95E1F78091A91931
:104F2000280F311D2655364EE091A519F091A6198E
:104F3000E90FF11DC901BF0150E00E94084DCD2BC2
:104F4000C9F08091AC1E9091AD1E892B31F48091F7
:104F5000A9198093AC1E1092AD1E2091A8198091C2
:104F6000AC1E9091AD1E820F911D9093AD1E80934B
:104F7000AC1E0BC02091A9198091A81990E0820F56
:104F8000911D9093AB1E8093AA1E2091AC1E309170
:104F9000AD1E2115310539F08091AA1E9091AB1EEE
:104FA00028173907F1F423ED32E2EAEAF9E14091FA
:104FB000AA1E5091AB1EC901BF010E94084D8091ED
:104FC000AA1E9091AB1E90935B2280935A2210925E
:104FD000AB1E1092AA1E1092AD1E1092AC1E0E9423
:104FE000360ADF91CF911F910895EF92FF920F93B0
:104FF0001F93CF93DF93182FE62EF42E052F80E01A
:1050000061E00E94650280E06E2D0E94650280E0F2
:10501000612F0E9465022F2D302FC901EC0104C0C1
:10502000699180E00E9465029E012F192E15C0F340
:1050300080E064E00E946502DF91CF911F910F91A3
:10504000FF90EF9008950F931F93CF93DF93EC01A0
:1050500088819981009729F08350914009F018C107
:105060004EC080E291E0909386218093852184E078
:1050700090E290938821809387218FE59FEF909312
:105080008A218093892180E09DE790938C218093F1
:105090008B2182E090ED90938E2180938D2187EB80
:1050A0009FEF9093902180938F218EEF93E29093C6
:1050B00092218093912186EE9BED90939421809391
:1050C000932185E891E260EF70EB40E050E00E94B0
:1050D000BC0CFC019093D11E8093D01E80EF91EB0D
:1050E000918B808B80E090E00E94B009882309F0CA
:1050F000CFC083E091E09983888381E0CCC06038A1
:1051000029F0613841F06130A1F70CC081EC60E01A
:1051100040E050E004C080EC61E04FEC5EE10E94B2
:10512000F527E7CF8091DD1E882319F38091DC1EDF
:10513000803809F481C0813809F0A7C08091D21E5F
:105140008093CF1E80E291E09093962180939521E9
:1051500084E090E290939821809397218FE59FEFD0
:1051600090939A218093992180E09DE790939C21D0
:1051700080939B2182E090ED90939E2180939D21CE
:1051800087EB9FEF9093A02180939F218EEF93E276
:105190009093A2218093A12186EE9BED9093A42170
:1051A0008093A32180E68093D3226093D42210922F
:1051B000D6221092D5228AE38093D9228091F020C2
:1051C0008093DA22ABEEB2E2E5E9F1E280E1019010
:1051D0000D928150E1F78BED92E26BEE72E20E944C
:1051E000B41AE091C520F0E08F0105501D4D80E814
:1051F000D8018C9311961C921197E150FD4D1082AD
:1052000011821282138280E390E090935B2280935C
:105210005A221092D72288E08093D82213961C92AB
:105220001E9212970E949D3980959095F801938364
:1052300082830E945C0A29C000D000D000D0EDB764
:10524000FEB7319605EA11E2ADB7BEB712961C93D0
:105250000E9311978FEB91E09383828382ED9EE111
:10526000958384830E94654DEDB7FEB736960FB6E1
:10527000F894FEBF0FBEEDBF8091D01E9091D11E5D
:10528000B80144E150E00E9458441092DD1E31CF35
:105290001982188283E0DF91CF911F910F910895B9
:1052A000282F8091DA1E813051F0813018F0823041
:1052B00061F408C01092DD1E213041F522C0209318
:1052C000DB1E1FC02093DC1E1CC0E82FF0E0809185
:1052D000DB1E90E002968E179F0784F4243059F469
:1052E00081E08093DD1E81EE91E061E040E050E0DE
:1052F0000E94790706C01092DA1E03C0E153F14EF6
:1053000020838091DA1E8F5F8093DA1E80E090E028
:10531000089587EE9EE108958091E61E089580919C
:10532000E41E089580E01B9981E0089529982B9848
:105330008CE090E00197F1F7299A0895DF92EF92BF
:10534000FF920F931F93DF93CF9300D00F92CDB7AF
:10535000DEB70091660080E88093660010927000CE
:1053600010926F008091B60080628093B6008091A9
:10537000B6008B71E1F781E08093B1008FB789832C
:10538000F89410E8DD24D39480E8E82EFF24FA9402
:10539000D09281008091B6008B71E1F7E092B2006B
:1053A0001092850010928400F7BAB89BFECF8091CE
:1053B0008400909185009B838A83109281006A818A
:1053C0007B8180E090E00E942C4A20E03FEE47EE97
:1053D00056E40E94A849882324F4809166008F5FD8
:1053E00013C06A817B8180E090E00E942C4A20E813
:1053F0003CE240E057E40E944849181614F081E06E
:1054000006C08091660081508093660080E0115054
:1054100021F0882309F4BCCF04C0882311F4009341
:1054200066001092B1008091B6008F7D8093B60027
:1054300089818FBF0F900F900F90CF91DF911F91B7
:105440000F91FF90EF90DF900895282F8EE268E093
:1054500043E00E94D92F0895882329F085E060E871
:1054600047E021E004C085E060E847E020E00E94DA
:10547000D92F08952B988CE090E00197F1F782E006
:105480006FE140E023E00E94D92F82E090E0019795
:10549000F1F708951F93162F603118F022E430E0E1
:1054A0001AC01B9B03C024E430E015C0882329F0F8
:1054B00081E160E144E021E004C081E160E144E099
:1054C00020E00E94D92F81E16FE040E0212F0E946F
:1054D000D92F20E430E0C9011F9108951F93282F90
:1054E000162F8330A8F4603198F41B9B03C024E48A
:1054F00030E010C088E060E645E00E94D92F89E0E6
:105500006FE040E0212F0E94D92F20E430E002C05C
:1055100022E430E0C9011F910895282F803118F04E
:1055200022E430E00CC01B9B03C024E430E007C041
:1055300085E06FE040E00E94D92F20E430E0C9010F
:1055400008950F931F93082F162F1B9B03C024E46D
:1055500030E02BC08CE260EF44E020E00E94D92FC5
:10556000212F30E02873307093E0359527959A9578
:10557000E1F78CE26EE041E00E94D92F212F2295C5
:105580002695269523708EE260EC46E00E94D92F86
:105590008DE2602F0E94AB2F17708EE267E040E033
:1055A000212F0E94D92F20E430E0C9011F910F91D3
:1055B0000895AF92BF92CF92DF92EF92FF920F9336
:1055C0001F938C017C010894E11CF11C84E2F8011A
:1055D00060810E94AB2F67010894C11CD11C85E239
:1055E000F80161810E94AB2F56010894A11CB11CE7
:1055F00086E2F70161810E94AB2F75010894E11CDE
:10560000F11C87E2F60161810E94AB2F87010F5FD9
:105610001F4F88E2F50161810E94AB2F89E2F701FB
:1056200061810E94AB2F8AE2F80161810E94AB2F59
:105630008BE20F5F1F4FF80161810E94AB2F1F911A
:105640000F91FF90EF90DF90CF90BF90AF900895B3
:105650001F93682F192F80E20E94AB2F81E2612FE8
:105660000E94AB2F1F9108951F93682F192F82E27C
:105670000E94AB2F83E2612F0E94AB2F1F910895F0
:10568000EF92FF920F931F937C0184E20E94902F70
:10569000F70181938F0185E20E94902FF7018183AA
:1056A00078010894E11CF11C86E20E94902FF80119
:1056B000818387010F5F1F4F87E20E94902FF701C0
:1056C000818378010894E11CF11C88E20E94902FEC
:1056D000F801818387010F5F1F4F89E20E94902F9D
:1056E000F70181838AE20E94902FF80181838BE287
:1056F0000E94902F0F5F1F4FF80181831F910F9120
:10570000FF90EF9008951F9381E20E94902F182F31
:1057100081E20E94902F512F40E0282F30E0242B6F
:10572000352BC9011F9108951F9383E20E94902F8A
:10573000182F82E20E94902F512F40E0282F30E056
:10574000242B352BC9011F9108958EE268E043E0B8
:105750000E94C62F089581E06FE140E00E94C62FAD
:1057600008951B9904C020E430E0C90108952B98E6
:1057700080EE96E00197F1F781E06FE140E00E9452
:10578000C62F883081F323E430E0EFCF1B990DC0A2
:105790000E943A2A81E06FE140E00E94C62F8830E3
:1057A00019F023E430E003C02B9A20E430E0C90173
:1057B00008950F931F93082F883059F0863049F0D1
:1057C000893039F0863129F0893119F022E430E04E
:1057D00056C01B9B03C024E430E051C081E06FE160
:1057E00040E00E94C62F182F81518230B8F311304B
:1057F000A9F3123099F3011709F43FC0083019F4E6
:105800000E943A2A26C0093139F4163199F482E00F
:105810006FE140E029E008C0063161F4193151F42C
:1058200082E06FE140E026E00E94D92F82E090E024
:105830000197F1F782E06FE140E0202F0E94D92F1D
:10584000183019F488E691E002C082E090E00197F8
:10585000F1F781E06FE140E00E94C62F801719F058
:1058600023E430E00CC0063011F0063121F481E071
:105870008093E51E02C01092E51E20E430E0C901CD
:105880001F910F91089581E06FE140E00E94C62FC3
:105890008850823018F024E430E016C088E160E8D7
:1058A00047E021E00E94D92F82E390E00197F1F7D1
:1058B00088E160E847E00E94C62F882319F420E4BD
:1058C00030E002C023E430E0C901089583E067E0DE
:1058D00040E00E94C62F08950F931F93082F162FA4
:1058E000663018F022E430E01CC083E067E040E05E
:1058F0000E94C62F811799F0002329F483E068E005
:1059000043E021E004C083E068E043E020E00E943F
:10591000D92F83E067E040E0212F0E94D92F20E4B7
:1059200030E0C9011F910F910895DF92EF92FF922D
:105930000F931F93D0906600F89481E061E00E947D
:105940006C2CE090B100F0908100009180001092EA
:10595000B100109281001092800020E030E04FEF03
:1059600063E056E046BB47BB1092B2001092850040
:10597000109284006093B10050938100B89BFECFD9
:10598000109281001092B100809184009091850066
:1059900073E08A3F970720F480916600815008C029
:1059A0008650944010F411E00CC0809166008F5F27
:1059B000809366002F5F3F4F83E0283E380791F6C3
:1059C00010E081E060E00E946C2CE092B100F09267
:1059D000810000938000112311F4D0926600812F82
:1059E0001F910F91FF90EF90DF90089581E160E2A9
:1059F00045E00E94C62F882319F02BE430E002C056
:105A00002AE430E0C901089581E160E144E00E94A8
:105A1000C62F089581E16FE040E00E94C62F0895EF
:105A2000CF93DF93EC0181E06FE140E00E94C62F4D
:105A3000863029F0813019F024E430E008C086E097
:105A40006FE140E00E94C62F888320E430E0C90166
:105A5000DF91CF91089589E06FE040E00E94C62F6A
:105A6000089588E060E645E00E94C62F089585E02D
:105A70006FE040E00E94C62F089588E06FE140E0AB
:105A80000E94C62F08951F93182F8B50803118F055
:105A900022E430E02BC01B9B03C024E430E026C08E
:105AA00088E06FE140E00E94C62F8117E9F088E0AE
:105AB0006FE140E0212F0E94D92F81E06FE140E0AB
:105AC0000E94C62F863011F0893021F48CE291E0DB
:105AD0000197F1F788E06FE140E00E94C62F81173F
:105AE00019F023E430E002C020E430E0C9011F9146
:105AF0000895DF92EF92FF920F931F937B018C0129
:105B0000D42E86E06FE140E00E94C62F8093E41E11
:105B1000E091DE1EF091DF1E309721F0C801B70141
:105B20004D2D09951F910F91FF90EF90DF900895F3
:105B30001F93CF93DF93182FEB0187FF03C022E45D
:105B400030E01FC081E06FE140E00E94C62F82304C
:105B5000B1F081E06FE140E00E94C62F823179F020
:105B600088E00E94D92B89E10E94D92B2B9A2B988F
:105B7000CE01612F0E94B43020E430E002C024E462
:105B800030E0C901DF91CF911F91089581E06FE16D
:105B900040E00E94C62F893019F024E430E029C08B
:105BA0008BE160E847E021E00E94D92F8AE160E8BC
:105BB00047E021E00E94D92F0E94802F8CE291E0E3
:105BC0000197F1F70E947D2F882389F08BE160E82F
:105BD00047E00E94C62F882351F48AE160E847E03D
:105BE0000E94C62F882319F420E430E002C023E489
:105BF00030E0C9010895CF92DF92EF92FF920F93A8
:105C00001F93CF93DF938B017A016901ECEFF3E0EF
:105C10003197F1F7882311F00E949E290E94C82E27
:105C200029982B988CE090E00197F1F7299A82E06F
:105C30006FE140E023E00E94D92F8CEF93E00197C1
:105C4000F1F781E06FE140E00E94C62F883019F043
:105C5000C3E4D0E014C08DE10E94902F81508230C7
:105C600060F48EE10E94902F8F3139F48EE06CE069
:105C70000E94AB2FC0E4D0E002C0C1E4D0E010939A
:105C8000DF1E0093DE1EF092E11EE092E01E89E727
:105C90009DE20E94592F8DE59EE20E94302FD09206
:105CA000E31EC092E21ECE01DF91CF911F910F91B2
:105CB000FF90EF90DF90CF900895DF93CF9300D0C7
:105CC00000D00F92CDB7DEB79B01AC01E091E01E92
:105CD000F091E11E309711F0099552C08091E51EB8
:105CE0008823C1F020937B1F30937C1F40937D1F3E
:105CF00050937E1F8091E41E80937A1F86EE9EE172
:105D000060E070E00E940E3086EE9EE168E67FE182
:105D10000E94E2318091E51E882391F588E00E947F
:105D2000D92B8091EB010E94D92B1B821A821D82F4
:105D30001C8282E060EE45E00E94C62F8983898143
:105D4000833059F0843018F4823058F403C0853021
:105D500041F403C081E190E002C082E190E09B83C6
:105D60008A838A819B81892B21F0CE0102960E9431
:105D700001034C815D8188E891E06A810E94790786
:105D80000F900F900F900F900F90CF91DF9108958B
:105D9000DF93CF930F92CDB7DEB71092811F109291
:105DA000801F8FB78983F8941092821F1092831FEF
:105DB0001092851F1092841F1092871F1092861FC9
:105DC00089818FBF239A219A84B1806B84B985B170
:105DD000806985B980E58CBD81E08DBD83E48093C9
:105DE0008100B59AEFE6F0E0808181608083808158
:105DF000806280830F90CF91DF910895DF93CF93DE
:105E00000F92CDB7DEB78FB78983F8941092821FB7
:105E10001092831F1092851F1092841F1092871F6B
:105E20001092861F89818FBF0F90CF91DF910895C7
:105E30008091821F0895DF93CF930F92CDB7DEB785
:105E40008FB78983F8941092821F89818FBF0F903A
:105E5000CF91DF9108958091861F9091871F0895BB
:105E6000DF93CF930F92CDB7DEB72FB72983F89486
:105E70009093871F8093861F89818FBF0F90CF914A
:105E8000DF910895DF93CF930F92CDB7DEB78FB731
:105E90008983F8941092871F1092861F89818FBF83
:105EA0000F90CF91DF9108958091841F9091851F6D
:105EB0000895DF93CF930F92CDB7DEB72FB7298325
:105EC000F8949093851F8093841F89818FBF0F90D2
:105ED000CF91DF910895DF93CF930F92CDB7DEB7C7
:105EE0008FB78983F8941092851F1092841F89813F
:105EF0008FBF0F90CF91DF9108958091831F0895F8
:105F0000DF93CF930F92CDB7DEB78FB78983F89425
:105F10001092831F89818FBF0F90CF91DF910895D9
:105F2000DF93CF930F92CDB7DEB780689FB7998389
:105F3000F8942C988EBD0DB407FEFDCF8EB58EBDA6
:105F40000DB407FEFDCF8EB52C9A99819FBF0F909F
:105F5000CF91DF910895DF93CF930F92CDB7DEB746
:105F6000806C9FB79983F8942C988EBD0DB407FE72
:105F7000FDCF8EB56EBD0DB407FEFDCF8EB52C9A4C
:105F800089818FBF0F90CF91DF910895FF920F937A
:105F90001F93062FF42E0E94902F082310E002C0BA
:105FA00015950795FA94E2F7802F1F910F91FF90B6
:105FB0000895EF92FF920F931F93DF93CF930F9269
:105FC000CDB7DEB7182F062FE42EF22E0E94902FA9
:105FD000282F106C8FB78983F8942C981EBD0DB4B0
:105FE00007FEFDCF8EB58F2D90E002C0880F991F60
:105FF000EA94E2F7802300950223802B8EBD0DB436
:1060000007FEFDCF8EB52C9A89818FBF0F90CF915F
:10601000DF911F910F91FF90EF9008958F929F92C3
:10602000AF92BF92CF92DF92EF92FF920F931F93A6
:10603000DF93CF930F92CDB7DEB78C014B01009762
:1060400021F46115710509F481C08FB78983F89433
:106050002C9880E28EBD0DB407FEFDCF8EB58EBDAF
:106060000DB407FEFDCFEEB48E2D83508D3708F0B2
:1060700060C00115110539F068010894C11CD11CDC
:10608000F801E08206C08E2D90E0F4010995CC2441
:10609000DD24EEBC0DB407FEFDCFAA24BB24FEB464
:1060A0001EBC0115110521F0F601F1926F0104C02B
:1060B0008F2D90E0F4010995C5018F25082E82955A
:1060C000807F8025092E982F82958F7008268695CF
:1060D00098278927880F880F880F80255C010DB4C9
:1060E00007FEFDCFEA94D9F60115110541F08EB5F2
:1060F00000581F4FF80180830058104004C08EB52F
:1061000090E0F40109952C9A0115110549F0F80168
:10611000EF57FF4F1082AB28B9F481E0808314C0A1
:1061200080E090E0AB2811F081E090E0F401099567
:106130000BC02C9A0115110539F0F8011082005896
:106140001F4FF8011192108289818FBF0F90CF915C
:10615000DF911F910F91FF90EF90DF90CF90BF9054
:10616000AF909F908F900895DF93CF930F92CDB70C
:10617000DEB7FC016F778FB78983F8942C9880E69F
:106180008EBD0DB407FEFDCF8EB56EBD0DB407FEFE
:10619000FDCF8EB581918EBD61500DB407FEFDCF50
:1061A0008EB56623B9F72C9A89818FBF0F90CF9156
:1061B000DF910895DF93CF930F92CDB7DEB7982F7D
:1061C000FA018FB78983F8942C981EBC0DB407FE92
:1061D000FDCF8EB59EBD0DB407FEFDCF8EB51EBCA6
:1061E0000DB407FEFDCF8EB58083615011F031965E
:1061F000F6CF2C9A89818FBF0F90CF91DF910895B0
:10620000DF93CF930F92CDB7DEB7982FFA018FB7F8
:106210008983F8942C9880E48EBD0DB407FEFDCFE1
:106220008EB59EBD0DB407FEFDCF8EB581918EBD9E
:106230000DB407FEFDCF8EB56150C1F72C9A898150
:106240008FBF0F90CF91DF9108951F920F920FB6DD
:106250000F920BB60F9211240F931F932F933F931E
:106260004F935F936F937F938F939F93AF93BF935E
:10627000EF93FF93DF93CF930F92CDB7DEB780916B
:10628000801F9091811FA0E0B0E09C0111270027A2
:106290008091840090918500A0E0B0E0082B192B3C
:1062A0002A2B3B2B2C988FE88EBD3695279517957A
:1062B00007950DB407FEFDCF8EB58EBD0DB407FE5C
:1062C000FDCF9EB52C9A92FF18C0E091841FF091EB
:1062D000851F309709F447C02C9880E28EBD0DB41D
:1062E00007FEFDCF8EB58EBD0DB407FEFDCF4EB5BA
:1062F0002C9AC901B801099536C093FF0AC0E091F4
:10630000861FF091871F309771F1C901B801099577
:106310002AC096FD28C091FD26C090FF06C080913E
:10632000831F8F5F8093831F1EC097FF1CC08EE06A
:106330000E94902F982F8FB78983F8942C988EEC19
:106340008EBD0DB407FEFDCF8EB59F779EBD0DB4FB
:1063500007FEFDCF8EB52C9A89818FBF8091821F59
:106360008F5F8093821F0F90CF91DF91FF91EF910C
:10637000BF91AF919F918F917F916F915F914F915D
:106380003F912F911F910F910F900BBE0F900FBE59
:106390000F901F9018951F920F920FB60F92112415
:1063A0008F939F938091801F9091811F019690936E
:1063B000811F8093801F9F918F910F900FBE0F9030
:1063C0001F9018950F931F93DF93CF93CDB7DEB730
:1063D00028970FB6F894DEBF0FBECDBF8C01DB014E
:1063E00057968C91579781FF19C08091881F8823F9
:1063F00089F485E190E09A8389831C821B82CE0117
:1064000001960E9401034B815C8188E891E06981DB
:106410000E94790781E08093881F9BC0A8014F5F8D
:106420005F4F11965C934E930D5F1F4F13961C9315
:106430000E93129703501040F801818187708230CB
:1064400021F450961C92509765C098012C5F3F4FE5
:10645000882331F115963C932E93149798012A5F67
:106460003F4F17961C921E921697FA0181818695CE
:1064700086958E5F8370823098F417963C932E93A6
:1064800016978181869586958370823021F49801D4
:10649000285F3F4F05C0833019F49801225F3F4FBA
:1064A00019961C921E921897F801818186FD07C0EB
:1064B00019963C932E9318972E5F3F4F08C0149661
:1064C0008D919C91159719969C938E9318971B9676
:1064D0003C932E931A97FA01818182958695869531
:1064E0008370823019F42E5F3F4F04C0833011F463
:1064F000285F3F4F1D961C921E921C97F8018081C9
:106500008250840F821B50968C9350971F963C9319
:106510002E931E9700581F4FF801819151968C932E
:1065200051978081817057962C9157972E7F282BF9
:1065300080E190E09E838D83B887AF832260579679
:106540002C93CE0105960E94010388E891E00E94F9
:10655000D90728960FB6F894DEBF0FBECDBFCF91F6
:10656000DF911F910F910895CF92DF92FF920F93C9
:106570001F93DF93CF9300D000D00F92CDB7DEB73B
:106580008C016B01FE01319685E0DF011D928A9539
:10659000E9F7F801218126952695237011F082E014
:1065A0008983D80111969C919295969596959370B2
:1065B00011F082E08B83291721F4F8018081806437
:1065C0008083D8018C9186FD1B82F801818186959C
:1065D0008695837090E08230910519F0039729F435
:1065E00002C082E001C088E08A83D80111968C91B4
:1065F000829586958695837090E08230910519F09A
:10660000039729F402C082E001C088E08C83F8017E
:10661000808183FF1DC087898695869586958370C6
:1066200090E08130910571F0823091051CF4892B46
:1066300039F00EC08230910539F0039749F406C055
:1066400085E005C086E003C08AE001C08EE08D834E
:10665000D8018D919C91119790938A1F8093891FE7
:1066600012968C9180938B1F8981823019F093E070
:10667000F92E09C0F8018381948190938D1F809336
:106680008C1F85E0F82E8A81823019F08830A1F5C0
:106690000DC0EF2DF0E0E757F04ED80115968D9123
:1066A0009C91169791838083B2E025C0EF2DF0E096
:1066B000E757F04ED80115968C9115978083169662
:1066C0008C911697818317968C91179782831896D1
:1066D0008C911897838319968C91199784831A96B5
:1066E0008C911A9785831B968C911B9786831C9699
:1066F0008C918783B8E0FB0E8B81823069F4EF2D9B
:10670000F0E0E757F04ED8011D968D919C911E97B1
:1067100091838083B2E0FB0E8C81823019F0883047
:10672000A1F50DC0EF2DF0E0E757F04ED8011F9610
:106730008D919C91509791838083B2E025C0EF2D7D
:10674000F0E0E757F04ED8011F968C911F97808399
:1067500050968C915097818351968C91519782835A
:1067600052968C915297838353968C91539784833E
:1067700054968C915497858355968C915597868322
:1067800056968C918783B8E0FB0EED81EE2379F06D
:106790002F2D30E02757304EA801495E5F4FC901C9
:1067A000BA014E2F50E00E94084D8D81F80E2F2D1A
:1067B00030E02757304EF80147A165A176A1C90105
:1067C00050E00E94084DD80197968C918E5F8F0DF6
:1067D000F601828389E89FE1918380830F900F9077
:1067E0000F900F900F90CF91DF911F910F91FF901D
:1067F000DF90CF9008959F92AF92BF92CF92DF9299
:10680000EF92FF920F931F93DF93CF93CDB7DEB735
:1068100028970FB6F894DEBF0FBECDBF81E00E946F
:1068200074038CE260EF44E022E00E94D92F8DECEB
:106830009BEA0E94342B1091BC21F090BD21E09086
:10684000BE21D090BF21C090C021B090C121A090A6
:10685000C2219090C3211983212F3F2D4E2D5D2DF4
:106860006C2D7B2D8A2D992D08E00E94F9452A83F5
:10687000212F3F2D4E2D5D2D6C2D7B2D8A2D992D99
:1068800000E10E94F9452B83212F3F2D4E2D5D2DD8
:106890006C2D7B2D8A2D992D08E10E94F9452C83C2
:1068A000212F3F2D4E2D5D2D6C2D7B2D8A2D992D69
:1068B00000E20E94F9452D83212F3F2D4E2D5D2DA5
:1068C0006C2D7B2D8A2D992D08E20E94F9452E838F
:1068D000212F3F2D4E2D5D2D6C2D7B2D8A2D992D39
:1068E00000E30E94F9452F83212F3F2D4E2D5D2D72
:1068F0006C2D7B2D8A2D992D08E30E94F945288760
:106900008CEB91E20E94D92A82ED94E00E94F04C37
:106910000E94EB4C8093B921A2E6B2E2ECEBF1E2EB
:1069200088E001900D928150E1F782E692E268E002
:106930000E94610328960FB6F894DEBF0FBECDBF4C
:10694000CF91DF911F910F91FF90EF90DF90CF904B
:10695000BF90AF909F9008959093BB218093BA21F0
:1069600008958091BA219091BB21089580930722C8
:1069700008958091072208952093FE213093FF21EE
:1069800040930022509301226093022270930322CD
:10699000809304229093052208952091FE21309146
:1069A000FF214091002250910122609102227091BA
:1069B0000322809104229091052208959093C7218B
:1069C0008093C62108958091C6219091C721089592
:1069D0002093F6213093F7214093F8215093F92129
:1069E0006093FA217093FB218093FC219093FD2109
:1069F00008952091F6213091F7214091F82150918E
:106A0000F9216091FA217091FB218091FC219091F4
:106A1000FD210895FC0184EC95E39183808381EC52
:106A200095E3938382838CEB95E39583848386EB54
:106A300095E3978386838CEA94E39187808781EB43
:106A400094E3938782878FEA95E39587848788EA22
:106A500095E39787868786EB94E3918B808B89EB10
:106A600094E3938B828B83E995E3958B848B8EE7FC
:106A700095E3978B868B87E795E3918F808F80E7EF
:106A800095E3938F828F8BE695E3958F848F84E6D1
:106A900095E3978F868F8CEB94E391A380A38DEC85
:106AA00094E393A382A38EED94E395A384A383EE52
:106AB00094E397A386A388EE94E391A780A789EF38
:106AC00094E393A782A708950E94A52B811181E0EA
:106AD000809306220895809306220E94252A089515
:106AE0000E94832B8093C4219093C52108958093A5
:106AF000C4219093C5210E94282B08958CEB91E22C
:106B00000E94402B2091BC213091BD214091BE219B
:106B10005091BF216091C0217091C1218091C2210B
:106B20009091C32108952093BC213093BD214093BF
:106B3000BE215093BF216093C0217093C1218093E7
:106B4000C2219093C3218CEB91E20E94D92A08952F
:106B50000E94942B8093F4219093F52108958093C3
:106B6000F4219093F5210E94342B08950E943D2D2D
:106B70008093082290E00895809308220E94432D7C
:106B800008950E94C62B08950E94B12B0895AC0170
:106B900020910F20822F90E04817590734F4241BCE
:106BA00020930F2021E030E004C010920F2020E05D
:106BB00030E0C901089540910B2050910C209C01B8
:106BC0004817590718F420E030E012C080910D20DA
:106BD00090910E20820F931F90930E2080930D2092
:106BE000421B530B50930C2040930B2021E030E0CC
:106BF000C901089590930C2080930B2008958091F3
:106C00000D2090910E20C0962091EC013091ED0165
:106C1000280F391FC901089580910F202091EC01A0
:106C20003091ED01280F311DC901089540E050E079
:106C30008091EC019091ED01C0962091102030914F
:106C400011202817390711F041E050E0CA010895DA
:106C50008091102090911120089580910B209091A7
:106C60000C20089590910F2080E3891B089580E304
:106C700090910F20891B20910B2030910C20280F20
:106C8000311DC9010895E82FF0E0EE0FFF1FE65D0A
:106C9000FD4D7183608381E090E00895E82FF0E07E
:106CA000EE0FFF1FE65DFD4D808191810895282F35
:106CB00030E043E0220F331F4A95E1F726593E4D5D
:106CC000C901089590E053E0880F991F5A95E1F7A4
:106CD00086599E4D0E94993781E090E00895EAE23E
:106CE000F2E21192119282E2E235F807D1F78AE0DE
:106CF00092E26EEE71E00E94993782E192E26EEECE
:106D000071E00E9499378AE192E26EEE71E00E9492
:106D1000993782E292E26EEE71E00E94993708950F
:106D200010920E2010920D2010920C2010920B2029
:106D300080E380930F208091EC019091ED01C0964B
:106D400090931120809310200E946F360895EF9247
:106D5000FF920F931F938C017B010E94903610933A
:106D6000112000931020F0920C20E0920B201F9134
:106D70000F91FF90EF900895AAE2B2E2FC0188E241
:106D800001900D928150E1F7AAE0B2E2FB0180E2AE
:106D900001900D928150E1F70895DC01EAE2F2E200
:106DA00088E201900D928150E1F7DB01EAE0F2E226
:106DB00080E201900D928150E1F70895EF92FF92E9
:106DC0000F931F937C0180910F2090E000E310E06F
:106DD000F801E81BF90B2091EC013091ED01280F2F
:106DE000391FC701B901AF010E94084D80910F20E2
:106DF000081B11090E0D1F1D20911020309111202C
:106E000080910D2090910E20280F391F40910B206A
:106E100050910C20C801B9010E94084D20910B200F
:106E200030910C20205D3F4F80910F20281B3109AD
:106E3000C9011F910F91FF90EF9008950F931F9339
:106E400040910F2050E000E310E0F801E41BF50B47
:106E50002091EC013091ED01240F351FB901AF01F4
:106E60000E94084D80910F20081B1109C8011F9135
:106E70000F910895E0911020F09111206091EC01A4
:106E80007091ED019B01205D3F4FE217F30749F040
:106E900040910B2050910C20C901BF010E94084D68
:106EA000089580910D2090910E200097D9F0409187
:106EB0000B2050910C20405D5F4FDC01D096A60F57
:106EC000B71F20E330E007C0FB01E20FF31F8D91F5
:106ED00080832F5F3F4F24173507B4F310920E20A5
:106EE00010920D200895EF92FF920F931F93F82EAA
:106EF000E92E162F072F0E949036212F302FC9011F
:106F00008C018138910510F000E810E0809110208C
:106F1000909111206F2D7E2DA8010E94084D109395
:106F20000C2000930B20C8011F910F91FF90EF9050
:106F30000895AC0120E030E0FA01E20FF31FDB011D
:106F4000A20FB31F8C9180832F5F3F4F28303105F4
:106F500099F70895AC0120E030E0FA01E20FF31F49
:106F6000DB01A20FB31F90818C91981719F020E0DC
:106F700030E007C02F5F3F4F2830310571F721E027
:106F800030E0C9010895AC0120E030E0F901EE5A8B
:106F9000FD4DDA01A20FB31F8C9180832F5F3F4F0D
:106FA0002830310599F70895FC0180819181228173
:106FB0003381820F931F918380830895EF92FF9214
:106FC0000F931F93FC01E080F180028113810E94E6
:106FD000D9000E0D1F1D081B190BC8011F910F9121
:106FE000FF90EF9008950F931F938C010E94D9009A
:106FF00040E050E0F80120813181821B930B228117
:1070000033818217930710F041E050E0CA011F91CD
:107010000F9108950F931F938C010E94D900F801DE
:10702000918380831F910F9108950F931F938C017B
:10703000FC01738362830E94D900F80191838083ED
:107040001F910F910895FC0180819181A281B381EC
:107050002481358146815781820F931FA41FB51F5C
:1070600080839183A283B3830895AF92BF92CF921E
:10707000DF92EF92FF920F931F93FC01A080B180EB
:10708000C280D380E480F580068117810E940F01C1
:10709000EA0CFB1C0C1D1D1DE61AF70A080B190B48
:1070A000B701C8011F910F91FF90EF90DF90CF9033
:1070B000BF90AF900895EF92FF920F931F938C01B2
:1070C0000E940F01E0E0F0E0D80114962D913D916F
:1070D0004D915C911797ED90FD900D911C91621B65
:1070E000730B840B950B6E197F09800B910B6F5FEF
:1070F0007F4F8F4F9F4710F4E1E0F0E0CF011F91E9
:107100000F91FF90EF9008950F931F938C010E94B1
:107110000F01F80160837183828393831F910F9124
:1071200008950F931F938C01FC014483558366835C
:1071300077830E940F01F8016083718382839383B8
:107140001F910F9108950E94EB4C08950E94F04CFE
:107150000895FC015381560F50936122272F332746
:107160004281420F40936022A181A0935F22E0817F
:10717000E0935E22842F90E08217930748F48A2FD1
:107180008F5F80935F22882319F4EF5FE0935E2284
:10719000852F90E070708617970790F4842F8F5F8B
:1071A00080936022882361F480915F228F5F8093B7
:1071B0005F22882329F480915E228F5F80935E2274
:1071C0000895FC0161507040680F791F20E030E0A5
:1071D0000EC0508140E08181DA01A80FB11D2A0F55
:1071E0003B1F2A173B0710F42F5F3F4F3296E617DD
:1071F000F70778F3E617F70749F4908180E0280F46
:10720000391F2817390710F42F5F3F4F832F922F14
:107210000895E3EDF2E240E050E0308120E081812A
:10722000B901680F711D460F571F4617570710F415
:107230004F5F5F4F329672E2EA3FF70770F382E2E8
:10724000EA3FF80751F4908180E0480F591F481732
:10725000590718F44F5F5F4F06C04115510519F4E7
:107260002FEF3FEF02C0342F252FC9010895CF9390
:10727000DF939091C520A92FB0E03091D72220E074
:107280002A1B3B0B9091D822290F311DA901480FD1
:10729000511DEBEDF2E2708160E08181EB01C80FDE
:1072A000D11D4C0F5D1F4C175D0710F44F5F5F4FF2
:1072B000329682E2EA3FF80770F382E2EA3FF8078B
:1072C00049F4908180E0480F591F4817590710F47E
:1072D0004F5F5F4FCD0185509D4D21503040280FAD
:1072E000391FFC010EC0708160E08181DB01A80FB5
:1072F000B11D4A0F5B1F4A175B0710F44F5F5F4FCA
:107300003296E217F30778F3E217F30751F490810E
:1073100080E0480F591F4817590718F44F5F5F4F17
:1073200006C04115510519F42FEF3FEF02C0342F6D
:10733000252FC901DF91CF9108958AE30E94373943
:10734000089586E00E943739089581E10E94373917
:1073500008950F931F93CF93DF93182F092F409118
:10736000C8205091C920BCE24F5F5F4F8DE740308D
:10737000580710F040E050E1342F252FA0E00EC058
:10738000AB9FF0011124ED58FD4D85A1882329F014
:10739000808991898217930739F3AF5FA23081F713
:1073A0004093C8205093C9201092C720E0E0F0E03D
:1073B00020E03CE21AC0239FD0011124AD58BD4DFE
:1073C00095968C919597882321F42093C720FD01F1
:1073D00010C0873049F4309731F096969C9196977B
:1073E00086A1891708F4FD012F5F223020F3209336
:1073F000C720309771F182E085A38091CA20808FE9
:107400008091CB20818F8091CC20828F8091CD2064
:10741000838F84EC94E0978F868F91A380A381E083
:1074200090E0958F848F17A281E086A383E084A3E8
:1074300012A280E183A3508B418B738B628BEF018F
:10744000212F302FC901DC0180E10D90099281507C
:10745000E1F7CF01DF91CF911F910F910895AC011A
:107460001092C72020E013C0E22FF0E0322F3F5FE0
:10747000EE0FFF1FE153FD4D808191818417950729
:1074800029F42093C720118210820895232F2230DF
:1074900058F32093C7200895AC011092C72020E034
:1074A00012C0E22FF0E0322F3F5FEE0FFF1FE153DB
:1074B000FD4D80819181892B29F42093C720518330
:1074C00040830895232F223060F32093C72008952E
:1074D000BC01809171229091722244960E94A93839
:1074E000E0917122F091722280915E22848B8091D2
:1074F0005F22858B80916022868B80916122878BB1
:107500000895282F892F922F0895EF92FF920F93BD
:107510001F939C0144275527F22EE32E00E010E034
:10752000362F272F40E050E0A90133272227E22AF7
:10753000F32A042B152BB701C8011F910F91FF905F
:10754000EF900895FC0140915C2250915D2223ED63
:1075500037E2241B350B621773070CF49B011216DC
:10756000130664F42093D5273093D627E417F50744
:1075700029F0CA01BF01A9010E94084D089582E0C7
:107580008093C620A091C5202A2F30E0F901E55054
:10759000FD4D8181682F70E0F3E0660F771FFA954B
:1075A000E1F7695F7F4F42E0285D3F4F3CC0F90142
:1075B000E80FF91FED52FD4D8081882319F08130CD
:1075C00019F42EC04F5F2FC090E0807C90708038FF
:1075D000910549F0803C910549F08034910501F511
:1075E0004093C62009C04093C62008C04093C620DF
:1075F0008091EB228F3F11F481E00895242F30E039
:1076000040E050E02A0F311D411D511D285D3F4FC4
:107610004F4F5F4F84E062E00E94BA4482E00895D9
:1076200081818E5F480F842F90E0681779070CF0F6
:10763000BECF4093C62080E008950F931F93CF9351
:10764000DF93C0917122D0917222843009F4A5C2D7
:107650000FE013E21093702200936F2210935D22CB
:1076600000935C22833099F48DA1282F30E02F7095
:1076700030702330310529F48C8D9D8D892B09F4D0
:1076800097C02230310511F00C94954380C08230B0
:1076900009F092C010925B2210925A221092D627C3
:1076A0001092D5278091CD208F5F8093CD208823A5
:1076B00099F48091CC208F5F8093CC20882361F453
:1076C0008091CB208F5F8093CB20882329F48091F9
:1076D000CA208F5F8093CA202DA1273011F025305A
:1076E00051F48EA18F5F8EA3883711F00C949543CF
:1076F0001DA20C949543222311F40C9495438C8D78
:107700009D8D892B09F450C08EA181508EA38F5F6F
:1077100011F00C9495433FA1383029F021502230CC
:1077200048F4353039F41DA280E880936A220E9423
:10773000EB09AAC6353010F080E307C083E090E083
:1077400002C0880F991F3A95E2F78EA38FA18F5F31
:107750008FA38DA190E08F70907083309105F1F030
:107760008430910544F48130910509F43BC40297BB
:1077700009F0DBC70CC08630910509F499C6883042
:10778000910509F495C6049709F0CFC791C6E09119
:10779000C520F0E0E550FD4D15862BC484E08093B4
:1077A0006A220E94EB09B2C62F70233009F0BDC7D0
:1077B00088E080936A225CC6853019F5E0916D22DD
:1077C000F0916E2280899189892B09F4AEC71092BD
:1077D000722210927122C8010C97909370228093AC
:1077E0006F2290935D2280935C221092D627109294
:1077F000D52710925B2210925A2288E080936A2249
:10780000CAC18091D322807F803609F08EC79091C3
:10781000D72280E02091D822AC01420F511D9A015D
:1078200080915A2290915B228417950708F47DC7B6
:10783000285D3F4F30935B2220935A228091DB22B8
:107840008F3F09F472C7C801849760E840E050E0B8
:107850000E94B01B892B09F044C0C80184970E9484
:10786000051C8823F1F58091EB228F3F09F05DC75D
:107870008091EC22823009F058C78091ED229091DE
:10788000EE22892B09F051C78091EF229091F022CE
:10789000892B09F04AC78091F1229091F222892B1D
:1078A00009F043C78091F3229091F422892B09F0CB
:1078B0003CC78091F5229091F622892B09F035C7BB
:1078C0008091F7229091F822892B09F02EC78091A0
:1078D000F922882309F029C78091FA22813009F022
:1078E00024C789ED92E290936C2280936B221092D0
:1078F000C5201092C420E0916B22F0916C2280810F
:107900008B3209F44BC08C3248F4863009F4B0C194
:10791000813109F4B4C0882389F06BC08A3309F43B
:1079200074C08B3320F48C3209F063C0FEC68B33F5
:1079300009F4FBC68C3309F05CC006C08091C420FA
:1079400080FD57C0816009C08091C42081FF04C0C0
:1079500086FD4FC0806401C082608093C4200E9475
:10796000BF3A813009F4E1C6813018F0823019F64F
:10797000E4C62091C520E22FF0E0CF0185509D4D57
:1079800090936C2280936B22285FFC018181880F89
:10799000880F880F280F2093C520ADCF8091C42079
:1079A00082FD27C084608093C4209091C520E92F78
:1079B000F0E0DF01A550BD4D13968C9113978823FD
:1079C00049F0BA969F01442737FD4095542F84E033
:1079D00060E018C0B0936C22A0936B22985FE550D2
:1079E000FD4D8181880F880F880F980F9093C520D7
:1079F00082CFE35DF2429F01442737FD4095542F2B
:107A000084E061E00E94BA4498C60E949D398F5F6D
:107A10009F4F09F08AC6E091C520F0E0E550FD4D8A
:107A200080810E94440AE091C520F0E0E550FD4DC0
:107A3000E081E538C1F0E63818F4E038A1F410C070
:107A4000E73829F0E73848F0E83869F403C00E94C5
:107A50008D180DC00E942C170AC00E945B1207C02F
:107A60000E948C4504C010925B2210925A22809191
:107A70005A2290915B22892B09F457C65EC68091E9
:107A80005A2290915B22C09790935B2280935A2256
:107A900083E093E29093702280936F22E091C5205F
:107AA000F0E0E550FD4D86819781892B31F00E94F1
:107AB000A5398F5F9F4F09F038C687ED97E2909305
:107AC0006E2280936D2248C028893989211531059D
:107AD000F1F18091C520E82FF0E0E550FD4D828165
:107AE00093818217930799F52A893B8921153105DE
:107AF00029F0808191818217930749F588819981C6
:107B0000892BE1F48A819B81892BC1F48C819D8131
:107B1000892BA1F48E819F81892B81F48885998599
:107B2000892B61F48A859B85892B41F48C859D8501
:107B3000892B21F48E859F85892BC1F08BED92E2F4
:107B4000BE0140E150E00E94FB4C009779F069963D
:107B5000D0936E22C0936D22C0916D22D0916E227F
:107B6000B8E2C930DB0708F4AFCFDFC5109272224C
:107B70001092712282E080936A2283E093E29093D4
:107B8000702280936F2290935D2280935C221092EA
:107B9000D6271092D5270E94EB092091D527309146
:107BA000D6272115310509F4C0C5C901C0969093A7
:107BB0005B2280935A22285F3F4F3093D72288520E
:107BC0008093D822A0916D22B0916E2254968C9110
:107BD00054978093DA2281E18093D922E091C520E5
:107BE000F0E0E550FD4D34832583178216825096D0
:107BF0008D919C9151979183808352968D919C9108
:107C0000539793838283ABEEB2E220916D22309141
:107C10006E22C901FC0180E101900D928150E1F7D3
:107C20008BED92E26BEE72E20E94B41A8FE093E267
:107C30009093702280936F228091C520C82FD0E04E
:107C4000C550DD4D0E94A539809590959F838E8308
:107C50008091C520E82FF0E0E550FD4D86819781A9
:107C6000892B09F058C58FEF9FEF9783868353C503
:107C70000E94A1398F5F9F4F09F057C58091C520A1
:107C8000082F10E005501D4DC3E7D2E28DA18823D7
:107C9000D9F0D80112962D913C9113978889998932
:107CA0002817390789F42D913C918A899B892817D7
:107CB000390751F48BED92E2BE0140E150E00E94A1
:107CC000FB4C009709F4B2C1AC96B2E2CF39DB07A6
:107CD000E9F2E0F2F80185858F73823001F5828147
:107CE00093819093D0208093CF201092C72013C00F
:107CF000E42FF0E0EE0FFF1FE153FD4D2091CF2068
:107D00003091D020808191812817390709F489C0EA
:107D10004F5F4093C7204091C720423048F3809185
:107D2000C520E82FF0E0DF01A550BD4D1D968C91D8
:107D30001D9782FDFAC484E11D968C931D978CE3F8
:107D400090E090935B2280935A22FD0180E5848726
:107D500097811B968C911B9717968C9317979387F7
:107D600096811A968C911A9716968C9316979287ED
:107D7000958119968C91199715968C9315979187E3
:107D800094819093C72018968C91189714968C9391
:107D9000149790871B968C911B978F5F1B968C93E3
:107DA0001B978823C1F41A968C911A978F5F1A96A5
:107DB0008C931A97882379F419968C9119978F5F71
:107DC00019968C931997882331F418968C911897EB
:107DD0008F5F18968C93E091C520F0E0DF01A550ED
:107DE000BD4D2D913C9111973093D0202093CF2001
:107DF000FD01828193819183808313963C932E931E
:107E00001297EBEEF2E2DF01509780E10D900192C4
:107E10008150E1F78BED92E26BEE72E20E94B41AB0
:107E200054C41092C720C0E0D0E04CE250E03CE2E5
:107E300025C0822F90E0849FF001859FF00D949FD4
:107E4000F00D1124ED58FD4D85A1882339F48CE205
:107E5000289FE0011124CD58DD4D14C0873059F41E
:107E6000209721F096A18EA1891728F4239FE00185
:107E70001124CD58DD4D2F5F2093C7202091C720BE
:107E80002230B8F2209709F450C4D0937222C093E4
:107E9000712283E08EA38CA31AA284E08BA31FA27D
:107EA000E091C520F0E0E550FD4D82819381998BF2
:107EB000888B808191819B8B8A8BDE01EBEDF2E2D6
:107EC00080E101900D928150E1F781E08DA38091D6
:107ED000CA20888F8091CB20898F8091CC208A8F77
:107EE0008091CD208B8F81E090E09D8F8C8FE091F1
:107EF000C520F0E0E550FD4D87818F8BE091C520D6
:107F0000F0E0E550FD4D86818E8BE091C520F0E0DC
:107F1000E550FD4D85818D8BE091C520F0E0E55069
:107F2000FD4D84818C8B81E090E00E94683AE09165
:107F3000C520F0E0E550FD4D848590E0807F907095
:107F4000813591050CF44EC01092C72035C0F9015F
:107F5000ED52FD4D84AD8093CE20882309F442C0BC
:107F6000813021F44F5F4093C72026C08230C1F496
:107F700085AD8430A9F436AD20E087AD90E0822B4A
:107F8000932B9093D0208093CF20F4E0853C9F07E3
:107F900010F084EC94E09F8F8E8F99A388A322C069
:107FA0008091C720E82FF0E0E05FFC4DE081EE23F8
:107FB000C9F0E80FE093C7204091C720242F30E09C
:107FC000E091C520F0E0E550FD4D848582958F70ED
:107FD00090E00597880F991F880F991F2817390778
:107FE0000CF4B5CFE091C520F0E0E550FD4D80E107
:107FF0008587E091C520F0E0DF01A550BD4D1D96BD
:108000008C911D9782601D968C931D97FD0182E0D7
:10801000848B84E0858B868B84EC878B80E490E076
:1080200090935B2280935A2280E60EC3D0937222F3
:10803000C093712210926A228091C520A82FB0E0CF
:10804000FD01E550FD4D858582FF03C01DA280E244
:1080500093C2848582958F70880F880F8093C72084
:1080600020915A2230915B2228523040281B31093E
:1080700030935B2220935A228DA18F70823039F485
:10808000A550BD4D1D968C918F73823139F1232BF4
:1080900059F4E091C520F0E0E550FD4D858590E074
:1080A00083709070892BD1F08091C520E82FF0E08B
:1080B000E550FD4D94818C89981709F0B2C29581E5
:1080C0008D89981709F0ADC296818E89981709F0AD
:1080D000A8C297818F89981709F0A3C2E091C520A3
:1080E000F0E0E550FD4D858584FF52C06C8D7D8D9F
:1080F0006115710509F44CC0CE0148960E94A9385B
:108100008091C520E82FF0E0E550FD4D208580915D
:108110005E222817E9F5918580915F229817C1F5B5
:10812000928580916022981799F5938580916122BC
:10813000981771F5288F80915F22898F8091602236
:108140008A8F809161228B8F8FA18823D1F42AA1FD
:108150009CA18EA1981B822F869586958695981B4B
:10816000392F320F3AA38BA1282F26952695821BF3
:1081700097FD9195890F8BA3369536953695830F8C
:108180008CA381E080936A228CA18EA31D8E1C8E0D
:108190008DA1282F30E0C9018F7090708430910537
:1081A00009F4EFC1853091055CF48230910591F1BD
:1081B000833091050CF0CAC0019709F0B6C210C017
:1081C0008630910509F425C2863091050CF4FDC175
:1081D0008730910509F425C2089709F0A6C2C6C1E7
:1081E00080916A2280FFA1C283E08DA380E4809306
:1081F0006A221D8E1C8E20915A2230915B222115FD
:10820000310509F431C182E480936A22C9010E94D8
:10821000683A2AC180916A2280FF8DC08091C52072
:10822000E82FF0E0E550FD4D85858F73823109F030
:1082300082C0848590E0807F9070813591050CF438
:108240004EC01092C72035C0F901ED52FD4D84ADEE
:108250008093CE20882309F442C0813021F44F5FFF
:108260004093C72026C08230C1F485AD8430A9F484
:1082700036AD20E087AD90E0822B932B9093D020F9
:108280008093CF2024E0853C920710F084EC94E0AA
:108290009F8F8E8F99A388A322C08091C720E82F3B
:1082A000F0E0E05FFC4DE081EE23C9F0E80FE093E1
:1082B000C7204091C720242F30E0E091C520F0E096
:1082C000E550FD4D848582958F7090E00597880F6D
:1082D000991F880F991F281739070CF4B5CF83E031
:1082E0008DA3E091C520F0E0E550FD4D84818C8B9D
:1082F000E091C520F0E0E550FD4D85818D8BE0914A
:10830000C520F0E0E550FD4D86818E8BE091C520C3
:10831000F0E0E550FD4D87818F8B81E090E00E9479
:10832000683A82E480936A221D8E1C8E10925B2232
:1083300010925A2299C080E280936A220E94EB092F
:10834000E0917122F091722215A2E9CC8091C520B2
:10835000E82FF0E0E550FD4D858580FF25C024FD28
:1083600023C08C8D9D8D892B09F0DFC180915A220D
:1083700090915B2201960E94683A20916A22822F96
:10838000806180936A2280915A2290915B22892B8E
:1083900019F0226120936A220E94EB0981E090E0AB
:1083A0009D8F8C8F88E082C085FF25C0328920E0B8
:1083B000838990E0282B392B80916F229091702235
:1083C000820F931F9093702280936F22E091C520BB
:1083D000F0E0E550FD4D328920E0838990E0282BC4
:1083E000392B80915A2290915B22821B930B9093A0
:1083F0005B2280935A2220915A2230915B222115D0
:10840000310559F08DA184FD08C080916A228260F7
:1084100080936A22C9010E94683AE091C520F0E089
:10842000E550FD4D968580E02785820F911D909344
:10843000D0208093CF2028A139A12817390710F028
:10844000892B21F43093D0202093CF208091CF200E
:108450009091D0209F8F8E8F80916A2290E08370C0
:108460009070892B09F461C11092D6271092D527FC
:108470000E94EB0980916A22282F85FF0CC0109280
:10848000D6271092D5271DA2E091C520F0E0E55037
:10849000FD4D84E1CCC084FF12C01092D62710920B
:1084A000D52781E090E09D8F8C8F84E08DA31FA263
:1084B000E091C520F0E0E550FD4D81E1B8C080912C
:1084C000D5279091D627892B01F120FF02C01D8E60
:1084D0001C8E8C8D9D8D0097A1F42E8D3F8D8091EB
:1084E000D5279091D6272817390720F43093D6271F
:1084F0002093D5278091D5279091D6279D8F8C8F5B
:1085000004C09093D6278093D5271FA280915C2228
:1085100090915D229093702280936F228091D52755
:108520009091D627892B81F08C8D9D8D009761F0DD
:10853000CC9690935B2280935A22E091C520F0E084
:10854000E550FD4D88E110C080916A2281FFEDC0A9
:108550008CE390E090935B2280935A22E091C520B7
:10856000F0E0E550FD4D80E1858768C080916A228A
:1085700080FFDBC01DA280E180936A220E94EB098C
:10858000D4C080915A2290915B22009711F00E94F2
:10859000683AE091C520F0E0E550FD4D8585909169
:1085A0006A2280FF0BC090FF06C087E08DA31EA249
:1085B0001D8E1C8E1DC086E08DA31AC090FF22C0A8
:1085C00085E08DA31D8E1C8EB0C080915A229091A3
:1085D0005B22009711F00E94683AE091C520F0E01C
:1085E000E550FD4D858580FF0DC087E08DA31EA25F
:1085F00081E090E00E94683A80E180936A220E94C4
:10860000EB090FC080915A2290915B22892B49F48B
:108610008CC080916A2280FF88C087E08DA31EA253
:1086200084C0E091C520F0E0E550FD4D80E18587F4
:108630008CE390E090935B2280935A22E091C520D6
:10864000F0E0E550FD4D80E58487E091C520F0E045
:10865000E550FD4D8C8980878D8981878E89828741
:108660008F898387888D8483898D85838A8D86838E
:108670008B8D878386E08093D9228889998991831D
:1086800080838A899B8993838283ABEEB2E2FE0169
:1086900080E101900D928150E1F78BED92E26BEE5B
:1086A00072E20E94B41A8DA1E091C52084FF06C039
:1086B000F0E0E550FD4D1786168607C0F0E0E55066
:1086C000FD4D84E0868784EC87878091F02080933D
:1086D000DA2280915A2290915B2288979093D72238
:1086E00080915A2288528093D822E091C520F0E0F0
:1086F0008F0105501D4DD80153961C9253975296E9
:108700001C92F801118A108A0E94A13980959095D7
:10871000F801918B808B80E68093D3221092D42233
:108720001092D6221092D52208C010925B2210928D
:108730005A221092C5201092C42010926A22DF9112
:10874000CF911F910F9108950F931F93CF93DF93B4
:108750008C014091C8205091C9204F5F5F4F8DE739
:108760004030580710F040E050E1342F252F809121
:10877000E7279091E8278217930779F380910028E3
:10878000909101288217930741F34093C82050939A
:10879000C9201092C72020E0A9E1B0E01CC0322F10
:1087A0003F5F822F90E08A9FF0018B9FF00D9A9F90
:1087B000F00D1124E952F84D80899189892B51F4EB
:1087C0002093C72089E1289FD0011124A952B84DD8
:1087D00049F427C0232F223010F32093C720A0E0B4
:1087E000B0E01FC050965C93509751964C935197B0
:1087F00053967C936E9352970115110531F480E1E5
:10880000ED0119928A95E9F707C0ED01F80180E1C1
:10881000019009928150E1F78091F02054968C9359
:108820005497CD01DF91CF911F910F9108950E9430
:10883000B81C0E94EF1180E009C0E82FF0E0EE0FB5
:10884000FF1FE153FD4D118210828F5F8230A8F32C
:1088500020E04CE250E00DC0822F90E0849FF001B8
:10886000859FF00D949FF00D1124ED58FD4D15A23C
:108870002F5F223088F380E094E09093C9208093AA
:10888000C82020E049E150E00EC0822F90E0849F94
:10889000F001859FF00D949FF00D1124E952F84DE1
:1088A000118A108A2F5F223080F32093C720089509
:1088B00090936E2280936D224093D5275093D627B4
:1088C000E3E0F3E29A0185E04130580714F020E03C
:1088D00035E0CF01A9010E94084D84E00E941D3BB4
:1088E0000E945C0A1092D6271092D5270895CF9245
:1088F000DF92EF92FF920F931F93DF93CF93CDB749
:10890000DEB760970FB6F894DEBF0FBECDBF7C0117
:10891000DE011196FC0180E101900D928150E1F79A
:10892000F701C288D388D701F90180E101900D9247
:108930008150E1F7F701138B028BC7010E94584465
:10894000D701FE01319680E101900D928150E1F74F
:10895000F701D38AC28A60960FB6F894DEBF0FBEC5
:10896000CDBFCF91DF911F910F91FF90EF90DF90DE
:10897000CF900895CF92DF92EF92FF920F931F93C3
:10898000CF93DF93D82EC62E79018A011092C5208D
:10899000A1EDB0E2EBEEF2E280E101900D928150A8
:1089A000E1F780915A2290915B22C09690935B22CE
:1089B00080935A228150954030F080E095E090936A
:1089C0005B2280935A2263ED72E240915A225091C9
:1089D0005B2240535040CB01C0960E94114D80E66F
:1089E0008093D3221092D4221092D6221092D522B4
:1089F0008AE38093D9228091F0208093DA228091BB
:108A0000DB229091DC22892B51F58091DD2290911F
:108A1000DE22892B21F58091DF229091E022892BA3
:108A2000F1F48091E1229091E222892BC1F48091AE
:108A3000E3229091E422892B91F48091E522909198
:108A4000E622892B61F48091E7229091E822892B1C
:108A500031F48091E9229091EA22892BD1F0EBEE5A
:108A6000F2E2DF01509780E10D9001928150E1F731
:108A70008091D1208F3F91F484E0D81651F422E008
:108A8000C21639F48BED92E261ED70E20E94B41AE5
:108A90000EC010925B2210925A2235C0ABEDB2E2AA
:108AA000E1EDF0E280E101900D928150E1F7E0917B
:108AB000C520CE2FD0E0FE01E550FD4DD082C18211
:108AC000C801B7010E94853AC150DD4D68837983A2
:108AD0008A839B8380915A2290915B2288979093FE
:108AE000D722889688528093D8228091C520C82F9B
:108AF000D0E0C550DD4D1B821A820E949D398095C1
:108B000090959B838A83DF91CF911F910F91FF9066
:108B1000EF90DF90CF90089523ED32E28091F02026
:108B20008093DA228091EB228F3F81F4D90158960D
:108B3000F901389680E101900D928150E1F78BEDBB
:108B400092E26BEE72E20E94B41A1BC0A1EDB0E299
:108B5000F901389680E101900D928150E1F7EBED3B
:108B6000F2E2DF01509680E10D9001928150E1F731
:108B7000ABEEB2E2E1EDF0E280E101900D928150C6
:108B8000E1F76091C520662301F18AE38093D92241
:108B900070E040915A2250915B22461B570B509334
:108BA0005B2240935A22485250405093D722485D4E
:108BB0005F4F842F88528093D82261507D4D4C5254
:108BC00050408FEF92E20E94114D1092C52081E833
:108BD0008093FB221092FC221092FE221092FD2222
:108BE0000E949D39809590959093FE228093FD225E
:108BF0000895EF92FF920F93DF93CF93CDB7DEB737
:108C000060970FB6F894DEBF0FBECDBFA82F00232C
:108C100009F461C07E010894E11CF11C88E0F701B1
:108C200011928A95E9F729833A834B835C836D839C
:108C30007E83AF83988780E2801BE82FFF27E7FDC4
:108C4000F0954D815E816F817885181684F01D86C0
:108C50001E861F86188A882799278E1B9F0B04C0A3
:108C600076956795579547958A95D2F728C0202F16
:108C7000332727FD3095DB01CA01022E04C0B695CB
:108C8000A795979587950A94D2F78D879E87AF878A
:108C9000B88B04C0440F551F661F771FEA95D2F7A3
:108CA00089819A81AB81BC8104C0B695A7959795BF
:108CB00087952A95D2F7482B592B6A2B7B2B49870E
:108CC0005A876B877C8729853A854B855C856D85BE
:108CD0007E85AF8598898A2F60960FB6F894DEBF9F
:108CE0000FBECDBFCF91DF910F91FF90EF90089510
:108CF000EF92FF920F931F937B018C0120E030E0F5
:108D000040E05FE40E94784988238CF0C801B701F5
:108D100020E030E040E05FE40E94F0470E94D84944
:108D20009B01AC01205030404040504806C0C80173
:108D3000B7010E94D8499B01AC01B901CA011F913A
:108D40000F91FF90EF900895A0E0B0E0EAEAF6E41A
:108D50000C949850DC012B01FA019C91923008F49C
:108D600039C1EB018881823008F433C1943069F451
:108D7000843009F02FC111969C9111978981981721
:108D800009F428C1A6EFB1E025C1843009F421C15E
:108D90008230A9F4923009F01DC19A01AD0188E03A
:108DA000EA010990AE01E90109929E018150C1F7E3
:108DB000E201898111969C918923818308C19230B7
:108DC00009F407C112962D903C901397EB018A810C
:108DD0009B811496AD90BD90CD90DC901797EC8060
:108DE000FD800E811F819101281B390BB90137FFCE
:108DF00004C066277727621B730B603271050CF085
:108E000061C0121613066CF537014801062E04C026
:108E100096948794779467940A94D2F721E030E08F
:108E200040E050E004C0220F331F441F551F6A95D5
:108E3000D2F721503040404050402E213F21402366
:108E40005123211531054105510521F021E030E084
:108E500040E050E079018A01E628F728082919291D
:108E60003CC0232BD1F1260E371E35014601062EBC
:108E700004C096948794779467940A94D2F721E07B
:108E800030E040E050E004C0220F331F441F551F64
:108E90006A95D2F721503040404050402A213B2172
:108EA0004C215D21211531054105510521F021E0BD
:108EB00030E040E050E059016A01A628B728C828F0
:108EC000D9280BC0821593052CF01C01AA24BB24C1
:108ED000650103C0EE24FF24870111969C91D20105
:108EE00011968C91981709F445C0992339F0A8017F
:108EF00097012A193B094C095D0906C0A601950195
:108F00002E193F09400B510B57FD08C011823382C7
:108F1000228224833583468357831DC081E0818369
:108F20003382228288279927DC01821B930BA40BB2
:108F3000B50B84839583A683B7830DC0220F331F9F
:108F4000441F551F24833583468357838281938131
:108F50000197938382832481358146815781DA0189
:108F6000C9010197A109B1098F5F9F4FAF4FBF435F
:108F700028F30BC0918333822282EA0CFB1C0C1D68
:108F80001D1DE482F5820683178383E0808324819C
:108F900035814681578157FF1AC0C901AA2797FD1D
:108FA000A095BA2F81709070A070B07056954795BB
:108FB00037952795822B932BA42BB52B84839583F0
:108FC000A683B78382819381019693838283DF0195
:108FD00001C0D201CD01CDB7DEB7E2E10C94B450AF
:108FE000A0E2B0E0E6EFF7E40C94A45069837A8342
:108FF0008B839C832D833E834F835887E9E0EE2E3D
:10900000F12CEC0EFD1ECE010196B7010E94C94B5A
:109010008E010F5E1F4FCE010596B8010E94C94B0D
:109020008A8991E089278A8BC701B801AE01475E22
:109030005F4F0E94A4460E94F44AA096E6E00C947A
:10904000C050A0E2B0E0E7E2F8E40C94A4506983D9
:109050007A838B839C832D833E834F835887F9E0EB
:10906000EF2EF12CEC0EFD1ECE010196B7010E94F1
:10907000C94B8E010F5E1F4FCE010596B8010E94AD
:10908000C94BC701B801AE01475E5F4F0E94A446BD
:109090000E94F44AA096E6E00C94C050A0E2B0E032
:1090A000E4E5F8E40C94985069837A838B839C837D
:1090B0002D833E834F835887CE010196BE01675FA3
:1090C0007F4F0E94C94BCE010596BE016F5E7F4F58
:1090D0000E94C94B9985923088F089898230C8F006
:1090E000943019F4823051F404C0843029F4923061
:1090F00081F486EF91E0C6C0923049F420E09A8571
:109100008A89981321E02A87CE010996BBC0823054
:1091100049F420E09A858A89981321E02A8BCE01B0
:109120004196B0C02D843E844F8458886D887E88D7
:109130008F88988CEE24FF248701AA24BB24650124
:1091400040E050E060E070E0E0E0F0E0C1018170FC
:109150009070892BE9F0E60CF71C081D191D9A0187
:10916000AB012A0D3B1D4C1D5D1D80E090E0A0E091
:10917000B0E0E614F7040805190520F481E090E05A
:10918000A0E0B0E0BA01A901480F591F6A1F7B1F78
:10919000AA0CBB1CCC1CDD1C97FE08C081E090E033
:1091A000A0E0B0E0A82AB92ACA2ADB2A3196E03228
:1091B000F10549F0660C771C881C991C569447945D
:1091C00037942794C3CFFA85EA892B893C898B850C
:1091D0009C85280F391F2E5F3F4F17C0CA01817031
:1091E0009070892B61F016950795F794E79480E0CD
:1091F00090E0A0E0B0E8E82AF92A0A2B1B2B76952C
:109200006795579547952F5F3F4F77FDE7CF0CC088
:10921000440F551F661F771F17FD4160EE0CFF1CA2
:10922000001F111F21503040403090E0590790E05E
:10923000690790E4790760F32B8F3C8FDB01CA014B
:109240008F779070A070B07080349105A105B10542
:1092500061F447FD0AC0E114F1040105110529F08C
:10926000405C5F4F6F4F7F4F40781A8EFE1711F0B2
:1092700081E08A8F4D8F5E8F6F8F78A383E0898F17
:10928000CE0149960E94F44AA096E2E10C94B450B3
:10929000A8E1B0E0EEE4F9E40C94A45069837A8389
:1092A0008B839C832D833E834F83588789E0E82EF0
:1092B000F12CEC0EFD1ECE010196B7010E94C94BA8
:1092C0008E010F5E1F4FCE010596B8010E94C94B5B
:1092D0008985823040F08989823028F0C701B80141
:1092E0000E94414C01C08FEF6896E6E00C94C0509C
:1092F000A8E1B0E0EEE7F9E40C94A45069837A8326
:109300008B839C832D833E834F83588789E0E82E8F
:10931000F12CEC0EFD1ECE010196B7010E94C94B47
:109320008E010F5E1F4FCE010596B8010E94C94BFA
:109330008985823040F08989823028F0C701B801E0
:109340000E94414C01C08FEF6896E6E00C94C0503B
:10935000A8E1B0E0EEEAF9E40C94A45069837A83C2
:109360008B839C832D833E834F83588789E0E82E2F
:10937000F12CEC0EFD1ECE010196B7010E94C94BE7
:109380008E010F5E1F4FCE010596B8010E94C94B9A
:109390008985823040F08989823028F0C701B80180
:1093A0000E94414C01C081E06896E6E00C94C050F8
:1093B000ACE0B0E0EEEDF9E40C94A85069837A8358
:1093C0008B839C83CE010196BE016B5F7F4F0E9411
:1093D000C94B8D81823061F1823050F1843021F4AB
:1093E0008E81882351F12EC02F81388537FD20C012
:1093F0006E812F3131051CF06623F9F023C08EE118
:1094000090E0821B930B29853A854B855C8504C0CF
:1094100056954795379527958A95D2F76623B1F0EB
:1094200050954095309521953F4F4F4F5F4F0EC05F
:1094300020E030E040E050E009C02FEF3FEF4FEF79
:109440005FE704C020E030E040E050E8B901CA0125
:109450002C96E2E00C94C450A8E0B0E0E2E3FAE419
:109460000C94A0507B018C0161157105810591055B
:1094700019F482E0898360C083E089838EE1C82E7D
:10948000D12CDC82CB82ED82FE820F831887C8014B
:10949000B7010E94A54AFC013197F7FF3BC0222784
:1094A00033272E1B3F0B57016801022E04C0D694B0
:1094B000C794B794A7940A94D2F740E050E060E0D4
:1094C00070E081E090E0A0E0B0E004C0880F991F58
:1094D000AA1FBB1F2A95D2F70197A109B1098E21B6
:1094E0009F21A023B1230097A105B10521F041E000
:1094F00050E060E070E04A295B296C297D294D83AA
:109500005E836F8378878EE190E08E1B9F0B9C8338
:109510008B8312C0309781F00E2E04C0EE0CFF1C1E
:10952000001F111F0A94D2F7ED82FE820F83188765
:10953000CE1ADF0ADC82CB821A82CE0101960E940B
:10954000F44A2896EAE00C94BC50EF92FF920F93F5
:109550001F937B018C0180E0E81680E0F80681E033
:10956000080780E0180788F48FEFE816F10401057A
:10957000110531F028F088E090E0A0E0B0E017C0DD
:1095800080E090E0A0E0B0E012C080E0E81680E06B
:10959000F80680E0080781E0180728F088E190E0ED
:1095A000A0E0B0E004C080E190E0A0E0B0E020E204
:1095B00030E040E050E0281B390B4A0B5B0B04C045
:1095C00016950795F794E7948A95D2F7F701E2503C
:1095D000FE4F8081281B310941095109C9011F91A2
:1095E0000F91FF90EF900895DF92EF92FF920F930B
:1095F0001F93FC01E480F58006811781D180808172
:10960000823048F480E090E0A0E1B0E0E82AF92A56
:109610000A2B1B2BA5C0843009F49FC0823021F493
:10962000EE24FF24870105C0E114F10401051105B2
:1096300019F4E0E0F0E096C0628173819FEF623838
:1096400079070CF05BC022E83FEF261B370B2A316D
:1096500031052CF020E030E040E050E02AC0B801B5
:10966000A701022E04C076956795579547950A94F1
:10967000D2F781E090E0A0E0B0E004C0880F991F2D
:10968000AA1FBB1F2A95D2F70197A109B1098E2104
:109690009F21A023B1230097A105B10521F081E00E
:1096A00090E0A0E0B0E09A01AB01282B392B4A2BC7
:1096B0005B2BDA01C9018F779070A070B070803495
:1096C0009105A105B10539F427FF09C0205C3F4F82
:1096D0004F4F5F4F04C0215C3F4F4F4F5F4FE0E063
:1096E000F0E02030A0E03A07A0E04A07A0E45A07E3
:1096F00010F0E1E0F0E079018A0127C060387105DF
:1097000064F5FB01E158FF4FD801C7018F779070D6
:10971000A070B07080349105A105B10539F4E7FE61
:109720000DC080E490E0A0E0B0E004C08FE390E0E2
:10973000A0E0B0E0E80EF91E0A1F1B1F17FF05C0CE
:1097400016950795F794E794319687E01695079557
:10975000F794E7948A95D1F705C0EE24FF2487019A
:10976000EFEFF0E06E2F679566276795902F9F7754
:10977000D794DD24D7948E2F8695492F462B582FCA
:109780005D29B701CA011F910F91FF90EF90DF9003
:109790000895FC01DB01408151812281622F6F77A6
:1097A00070E0221F2227221F9381892F880F822B8E
:1097B000282F30E0991F9927991F11969C93119794
:1097C00021153105A9F5411551056105710511F402
:1097D00082E037C082E89FEF13969C938E93129796
:1097E0009A01AB0167E0220F331F441F551F6A9592
:1097F000D1F783E08C930DC0220F331F441F551FF8
:1098000012968D919C911397019713969C938E932A
:109810001297203080E0380780E0480780E458073E
:1098200058F314962D933D934D935C931797089599
:109830002F3F310579F4411551056105710519F482
:1098400084E08C93089564FF03C081E08C9312C080
:109850001C9210C02F57304013963C932E931297B2
:1098600083E08C9387E0440F551F661F771F8A950E
:10987000D1F7706414964D935D936D937C93179715
:1098800008951F93DC01FB019C91923008F447C0BE
:109890008081823008F443C0943051F411961C91B9
:1098A000843099F58181682F70E0611B71093FC098
:1098B000843021F0923031F48230B9F181818823F3
:1098C00089F12DC011961C9111978230F1F08181A0
:1098D0001817D9F412962D913C9113978281938198
:1098E0008217930794F028173907BCF014968D91CE
:1098F0009D910D90BC91A02D248135814681578189
:10990000281739074A075B0718F4112341F00AC0EA
:1099100082179307A407B50740F4112319F061E0FB
:1099200070E005C06FEF7FEF02C060E070E0CB0138
:109930001F910895A0E0B0E0E0EAFCE40C94A05090
:10994000EC01A880B980CA80DB80A114B104C104F5
:10995000D10441F484E2A82E89EDB82E8BE5C82EFF
:1099600087E0D82EC601B5012DE133EF41E050E08C
:109970000E94CF5027EA31E440E050E00E9430508E
:109980007B018C01C601B5012DE133EF41E050E0D0
:109990000E94CF50CA01B9012CEE34EF4FEF5FEFB8
:1099A0000E9430506E0D7F1D801F911F97FF04C0D5
:1099B0006150704080409048688379838A839B839C
:1099C0009B013F77C901CDB7DEB7EAE00C94BC50EC
:1099D0000E949A4C08958EEF92E00E949A4C08954E
:1099E000A0E0B0E08093FE029093FF02A0930003FA
:1099F000B09301030895FB01DC0104C08D91019037
:109A0000801921F441505040C8F7881B990B0895E4
:109A1000FB01DC0102C001900D9241505040D8F78B
:109A200008956817790768F4FB01DC01E40FF51F5E
:109A3000A40FB51F02C002900E9241505040D8F7BB
:109A400008950C94084DA0E0B0E0E9E2FDE40C9428
:109A5000A2507C01EB018A01690109C0CE01219667
:109A6000F6010995F70181937F010150104001151E
:109A70001105A1F7CDB7DEB7E8E00C94BE50A0E029
:109A8000B0E0E5E4FDE40C94A850FE013596619148
:109A90007191A0910B28B0910C2813968C9113977B
:109AA000886013968C9380910B2890910C28AF01BD
:109AB0000E94B34DE0910B28F0910C282381277F61
:109AC00023832096E2E00C94C450AEE0B0E0EBE6D5
:109AD000FDE40C94A6500D891E8986E08C831A83C0
:109AE00009838FEF9FE79E838D839E01275E3F4F03
:109AF000CE0101966F89788DA9010E94B34D2F8107
:109B00003885020F131FF80110822E96E4E00C94A2
:109B1000C250AEE0B0E0EFE8FDE40C94A6508C013A
:109B200077FF02C060E070E8615070407E836D8313
:109B30001A83098386E08C83CE010196BA01A901BC
:109B40000E94B34D2D813E8137FD09C0EF81F8851C
:109B50002E173F070CF4F901E00FF11F10822E962B
:109B6000E4E00C94C250ABE0B0E0E9EBFDE40C940F
:109B700098503C012B015A01FC0117821682838107
:109B800081FD03C06FEF7FEFC6C19AE0892E1E01F1
:109B90000894211C311CF3012381F20123FD8591DE
:109BA00023FF81912F01882309F4B2C1853239F452
:109BB00023FD859123FF81912F01853229F490E0C7
:109BC000B3010E94A64FE7CF982FFF24EE249924DB
:109BD000FFE1FF15D0F09B3269F09C3228F49032FF
:109BE00059F0933291F40EC09D3249F0903369F4EC
:109BF00041E024C052E0F52A84E0F82A28C098E029
:109C0000F92A25C0E0E1FE2A22C0F7FC29C0892FED
:109C100080538A3070F4F6FE05C0989C902C112475
:109C2000980E15C0E89CE02C1124E80EF0E2FF2A03
:109C30000EC09E3229F4F6FC6BC140E4F42A07C042
:109C40009C3619F450E8F52A02C0983649F4F2011E
:109C500023FD959123FF91912F01992309F0B8CF0E
:109C6000892F8554833018F08052833038F444E0D3
:109C700050E0A40EB51E5FE359830FC0933631F058
:109C8000933779F0933509F056C020C0F5018081F3
:109C9000898342E050E0A40EB51E610101E010E0AE
:109CA00012C0F501C080D180F6FC03C06FEF7FEFDA
:109CB00002C0692D70E042E050E0A40EB51EC6015E
:109CC0000E949B4F8C015FE7F52214C0F501C08014
:109CD000D180F6FC03C06FEF7FEF02C0692D70E00A
:109CE00042E050E0A40EB51EC6010E94904F8C01C8
:109CF00050E8F52AF3FE07C01AC080E290E0B301F5
:109D00000E94A64FEA948E2D90E008171907A8F339
:109D10000EC0F601F7FC8591F7FE81916F0190E08E
:109D2000B3010E94A64FE110EA94015010400115C2
:109D3000110579F7EAC0943611F0993669F5F7FE06
:109D400008C0F501208131814281538184E090E097
:109D50000AC0F501808191819C01442737FD40951F
:109D6000542F82E090E0A80EB91E9FE6F92257FF1B
:109D700009C050954095309521953F4F4F4F5F4F0B
:109D8000E0E8FE2ACA01B901A1012AE030E00E9400
:109D9000D24FD82ED21840C0953729F41F2D1F7EE0
:109DA0002AE030E01DC01F2D197F9F3661F09037EB
:109DB00020F4983509F0ACC00FC0903739F09837CF
:109DC00009F0A6C004C028E030E00AC0106114FD0C
:109DD000146020E130E004C014FD166020E132E0A0
:109DE00017FF08C0F501608171818281938144E091
:109DF00050E008C0F50180819181BC0180E090E0D5
:109E000042E050E0A40EB51EA1010E94D24FD82E10
:109E1000D2188FE7F82EF122F6FE0BC05EEFF52286
:109E2000D91438F4F4FE07C0F2FC05C08FEEF82216
:109E300002C01D2D01C0192DF4FE0DC0FE01ED0D57
:109E4000F11D8081803319F499EEF92208C01F5F5B
:109E5000F2FE05C003C08F2D867809F01F5F0F2D1D
:109E6000F3FC14C0F0FE0FC01E1510F09D2C0BC0AB
:109E70009D2C9E0C911A1E2D06C080E290E0B3012D
:109E80000E94A64F1F5F1E15C0F304C01E1510F4DC
:109E9000E11A01C0EE2404FF0FC080E390E0B3019B
:109EA0000E94A64F02FF1DC001FD03C088E790E09D
:109EB0000EC088E590E00BC0802F867891F001FFFE
:109EC00002C08BE201C080E2F7FC8DE290E0B301BA
:109ED0000E94A64F06C080E390E0B3010E94A64F07
:109EE0009A94D914C0F3DA94F101ED0DF11D80813B
:109EF00090E0B3010E94A64FDD20A9F706C080E2E2
:109F000090E0B3010E94A64FEA94EE20C1F743CE41
:109F1000F30166817781CB012B96E2E10C94B4507A
:109F2000FC010590615070400110D8F78095909524
:109F30008E0F9F1F0895FC01615070400190011029
:109F4000D8F7809590958E0F9F1F08950F931F93BC
:109F5000CF93DF938C01EB018B8181FF1BC082FFCC
:109F60000DC02E813F818C819D812817390764F4B3
:109F7000E881F9810193F983E88306C0E885F985D2
:109F8000802F0995892B31F48E819F8101969F83C3
:109F90008E8302C00FEF1FEFC801DF91CF911F9199
:109FA0000F910895FA01AA27283051F1203181F14B
:109FB000E8946F936E7F6E5F7F4F8F4F9F4FAF4FD1
:109FC000B1E03ED0B4E03CD0670F781F891F9A1FE4
:109FD000A11D680F791F8A1F911DA11D6A0F711D98
:109FE000811D911DA11D20D009F468943F912AE0A4
:109FF000269F11243019305D3193DEF6CF0108958C
:10A00000462F4770405D4193B3E00FD0C9F7F6CFBC
:10A01000462F4F70405D4A3318F0495D31FD405284
:10A02000419302D0A9F7EACFB4E0A695979587951A
:10A0300077956795BA95C9F70097610571050895F9
:10A040009B01AC010A2E06945795479537952795A5
:10A05000BA95C9F7620F731F841F951FA01D08953D
:10A06000629FD001739FF001829FE00DF11D649FFC
:10A07000E00DF11D929FF00D839FF00D749FF00D88
:10A08000659FF00D9927729FB00DE11DF91F639F29
:10A09000B00DE11DF91FBD01CF0111240895AA1BC8
:10A0A000BB1B51E107C0AA1FBB1FA617B70710F0C3
:10A0B000A61BB70B881F991F5A95A9F780959095F5
:10A0C000BC01CD01089597FB092E07260AD077FD24
:10A0D00004D0E5DF06D000201AF4709561957F4F1B
:10A0E0000895F6F7909581959F4F0895A1E21A2E55
:10A0F000AA1BBB1BFD010DC0AA1FBB1FEE1FFF1F2C
:10A10000A217B307E407F50720F0A21BB30BE40B7B
:10A11000F50B661F771F881F991F1A9469F76095C2
:10A120007095809590959B01AC01BD01CF0108957C
:10A130002F923F924F925F926F927F928F929F9257
:10A14000AF92BF92CF92DF92EF92FF920F931F9345
:10A15000CF93DF93CDB7DEB7CA1BDB0B0FB6F894F6
:10A16000DEBF0FBECDBF09942A88398848885F8436
:10A170006E847D848C849B84AA84B984C884DF80A7
:10A18000EE80FD800C811B81AA81B981CE0FD11D8B
:10A190000FB6F894DEBF0FBECDBFED01089597FB5B
:10A1A000092E05260ED057FD04D0A0DF0AD0001CD2
:10A1B00038F450954095309521953F4F4F4F5F4F64
:10A1C0000895F6F790958095709561957F4F8F4F24
:08A1D0009F4F0895F894FFCFA2
:10A1D800496E697420737461636B2070726F636574
:10A1E80073730000000001790000000000130100F3
:10A1F80000000000000000436F6E74696B69203234
:10A208002E33009E018801B501E101000000000025
:10A218000200000000970200000000C600C500C44C
:10A2280000C100C200000000CE00CD00CC00C90073
:10A23800CA00000000C00300000000000000000089
:10A248000000003830322E31352E34204D41432065
:10A2580070726F636573730000007301B5050000C9
:10A2680000004576656E742074696D6572000000A3
:10A278009201B708000000005443502F4950207342
:10A288007461636B000000A8017B0B0000000054A0
:10A2980025730D0A00526176656E204C434420698F
:10A2A8006E746572666163652070726F636573733F
:10A2B800000000C50123280000000016122000003D
:10A2C8000000000000000000000000000000000185
:10A2D800020203030303040404040404040405053C
:10A2E8000505050505050505050505050505060614
:10A2F80006060606060606060606060606060606F6
:10A3080006060606060606060606060606060707E3
:10A3180007070707070707070707070707070707C5
:10A3280007070707070707070707070707070707B5
:10A3380007070707070707070707070707070707A5
:10A348000707070707070707070707070707080893
:10A358000808080808080808080808080808080875
:10A368000808080808080808080808080808080865
:10A378000808080808080808080808080808080855
:10A388000808080808080808080808080808080845
:10A398000808080808080808080808080808080835
:10A3A8000808080808080808080808080808080825
:10A3B8000808080808080808080808080808080815
:10A3C8000808080808080808080808080808010014
:00000001FF
